:020000040000FA
:1000000002EF00F00F01FF0E926E000E936E000ED5
:10001000946E000E956E0F0E966E030E386F000EE6
:10002000396F000E3A6F000E3B6F000E3C6F010EF1
:10003000C26E040EC16EB20EC06E700ED36E400E54
:100040009B6E806A816A826A836A846A896A8A6A24
:100050008B6A8C6A8D6A00018C8C006A016A026A64
:10006000036A046A056A066A076A086A096A0A6A0C
:100070000B6A0C6A0D6A0E6A0F6A106A116A126ABC
:10008000136A146A156A166A176A186A196A1A6A6C
:100090001B6A1C6A1D6A1E6A1F6A206A216A226A1C
:1000A000236A246A266A286A296A2A6A2B6A2C6AC1
:1000B0002D6A2E6A2F6A306A316A326A336A346A6C
:1000C000356A366A376A386A396A3A6A3E6A3F6A16
:1000D000406A416A426A436A446A456A466A476AB4
:1000E000486A496A4A6A4B6A4C6A4D6A8A848A82BB
:1000F000FF0E3D6EFF0E256EFF0E276EB3EC23F054
:10010000000EAA6E000EA96EA69EA69CA6800000F8
:100110000000A850366E000EAA6E010EA96EA69EB3
:10012000A69CA68000000000A850406E000EAA6E9B
:10013000020EA96EA69EA69CA68000000000A850F4
:100140004A6E36503F6E4050416E4A504B6E64ECE2
:100150001DF0DCEC1AF0C00E8B6E8C928C900000BF
:10016000000000000000000000008C84000000007F
:10017000000000000000000000000000000000007F
:10018000000000000000000000000000000000006F
:100190000000000000000000000000008C9400003F
:1001A000000000000000000000000000000000004F
:1001B000000000000000000000000000000000003F
:1001C0005DEC1BF03F0E8B6E8C928C90000000005B
:1001D00000000000000000008C840000000000000F
:1001E000000000000000000000000000000000000F
:1001F00000000000000000000000000000000000FF
:10020000000000000000000000008C9400000000CE
:1002100000000000000000000000000000000000DE
:10022000000000000000000000000000000046EC9C
:100230001CF08C8EDFEC1AF084EC1DF0C46AC36AEB
:1002400036AC53EF01F0000EAA6E030EA96EA69E07
:10025000A69CA68000000000A850256E000EAA6E85
:10026000040EA96EA69EA69CA68000000000A850C1
:10027000266E000EAA6E050EA96EA69EA69CA680EE
:1002800000000000A850276E000EAA6E060EA96E90
:10029000A69EA69CA68000000000A850286E9DEC9B
:1002A00023F0A8EC23F036A059EF01F08A965AEF1C
:1002B00001F08A867EEC21F080B47BEF01F00C0E19
:1002C000445CD8B467EF01F0442A7DEF01F0446A42
:1002D00011BA7DEF01F0118A36A076EF01F09DECA6
:1002E00023F0A8EC23F036907DEF01F0B3EC23F07F
:1002F00036807DEF01F0119A446A010EC26EC294FD
:10030000C282C2B281EF01F0000EC26EC4502B6EE9
:10031000C3502A6E7EEC21F0010EC26EC284C282EE
:10032000C2B290EF01F0C4502D6EC3502C6E000E7F
:10033000C26E7EEC21F0C8EC23F084B008EF02F02E
:100340000C0E475CD8B4A8EF01F0472A0AEF02F080
:10035000476A11B80AEF02F01188000E145CD8B495
:100360000AEF02F0010E145CD8B4C3EF01F0020EE4
:10037000145CD8B4D7EF01F0EDEF01F0146A46EC4D
:100380001CF00AEF02F012A0CBEF01F036503F6EE6
:1003900012900AEF02F0196A12A21A6A12A41B6ADA
:1003A000146A396A3A6A46EC1CF00AEF02F012A2AB
:1003B000E1EF01F04050416E4A504B6E12920AEF4D
:1003C00002F012A0196A1A6A12A41B6A146A396A26
:1003D0003A6A46EC1CF00AEF02F012A4FCEF01F0BE
:1003E0004390439236ACF8EF01F03F8CF9EF01F007
:1003F0003F9C12940AEF02F012A0196A12A21A6A24
:100400001B6A146A396A3A6A46EC1CF00AEF02F079
:100410001198476A36BA7EEC21F084B207EF03F0F8
:100420000C0E485CD8B418EF02F0482A09EF03F02C
:10043000486A11B609EF03F01186000E145CD8B4B7
:1004400009EF03F0010E145CD8B42EEF02F0020E97
:10045000145CD8B4A7EF02F0BCEF02F012B034EF96
:1004600002F0128009EF03F036A03AEF02F03F806D
:100470003BEF02F03F903F50366E010E195CD8A45E
:1004800072EF02F036B859EF02F036A64BEF02F0E9
:1004900036AA59EF02F0100E255CD8B459EF02F0DD
:1004A00026503F0B0008D8B459EF02F0266AA8EC9A
:1004B00023F036B89DEF02F036A662EF02F036AABE
:1004C000A4EF02F0100E275CD8B4A4EF02F028507D
:1004D0003F0B0008D8B4A4EF02F0286AA8EC23F080
:1004E000A4EF02F0020E195CD8A4A4EF02F036AA21
:1004F00087EF02F0100E255CD8B488EF02F026508A
:100500003F0B0008D8B488EF02F036A8266A269C74
:1005100036AA98EF02F0100E275CD8B499EF02F0DB
:1005200028503F0B0008D8B499EF02F036A8286A8B
:10053000289CA8EC23F0A4EF02F036A8A4EF02F068
:10054000269C289CA8EC23F0129009EF03F012B22D
:10055000ADEF02F0128209EF03F04150406E4B50B4
:100560004A6E2E6A2F6A306A316A326A336A346A96
:10057000356A129209EF03F012B4C2EF02F012844E
:1005800009EF03F0000E1B5CD8A4DFEF02F043A0DC
:10059000DCEF02F04390D6EC2EF0FDEC2EF010ECE8
:1005A0002FF036ACDCEF02F023EC2FF036EC2FF01E
:1005B00049EC2FF05CEC2FF0129409EF03F0020EDF
:1005C0001B5CD8A4FDEF02F043A2FAEF02F04392C5
:1005D000366A3F6A406A416A010E4A6E010E4B6EEE
:1005E000FF0E256EFF0E276E266A286A9DEC23F00B
:1005F000A8EC23F0129409EF03F03FAC03EF03F0F3
:10060000368C04EF03F0369C129409EF03F0119638
:10061000486A36BA7EEC21F084B42DEF03F00C0E5C
:10062000495CD8B417EF03F0492A2FEF03F0496A69
:1006300011B02FEF03F01180030E145CD8B426EF35
:1006400003F0142A46EC1CF02FEF03F0146A396A09
:100650003A6A46EC1CF02FEF03F01190496A000E45
:10066000145CD8B440EF03F0010E145CD8B4EBEF87
:1006700008F0020E145CD8B439EF10F0DDEF15F07D
:100680007EEC21F0D6EC1AF0410EE2EC1AF0B80E36
:100690000AEC1BF0700E32EC1BF0100E32EC1BF06B
:1006A000100E32EC1BF0100E32EC1BF0000E32EC90
:1006B0001BF03EEC2CF0000E32EC1BF0CEEC2BF0DD
:1006C000000E32EC1BF09EEC2BF0000E32EC1BF017
:1006D0002EEC2CF0000E32EC1BF0AEEC2BF0000EEA
:1006E00032EC1BF03EEC2BF04EEC2EF00EEC2CF02E
:1006F000000E32EC1BF01EEC2CF0000E32EC1BF066
:10070000FEEC2AF0D9EC1AF0400EE2EC1AF0B80E2A
:100710000AEC1BF01EEC2CF0000E32EC1BF02EEC61
:100720002CF0000E32EC1BF00EEC2CF0000E32EC34
:100730001BF0082A2D0E085CD8B4A4EF03F0100EAD
:1007400032EC1BF099EF03F0086A700E32EC1BF0EC
:10075000D6EC1AF0410EE2EC1AF0BB0E0AEC1BF0DC
:10076000700E32EC1BF0100E32EC1BF0100E32EC5F
:100770001BF0100E32EC1BF0000E32EC1BF09EEC66
:100780002BF04EEC2EF01EEC2BF0000E32EC1BF09A
:100790006EEC2BF0000E32EC1BF0082A230E085CE6
:1007A000D8B4D8EF03F0100E32EC1BF0CDEF03F00D
:1007B000086A700E32EC1BF0D9EC1AF0410EE2EC34
:1007C0001AF0BB0E0AEC1BF0700E32EC1BF0100E90
:1007D00032EC1BF0100E32EC1BF0100E32EC1BF062
:1007E000000E32EC1BF0FEEC2BF04EEC2EF01EEC6B
:1007F0002BF0000E32EC1BF06EEC2BF0000E32EC06
:100800001BF0082A230E085CD8B40CEF04F0100E7D
:1008100032EC1BF001EF04F0086A700E32EC1BF0B2
:100820007EEC21F0D6EC1AF0410EE2EC1AF0BC0E90
:100830000AEC1BF0FEEC2AF0000E32EC1BF072EC1E
:100840002EF0000E32EC1BF0000E32EC1BF02550A7
:10085000296EFF0E295CD8A452EF04F04EEC2EF066
:10086000000E32EC1BF0000E32EC1BF092EC2EF07E
:10087000000E32EC1BF092EC2EF0000E32EC1BF06E
:1008800092EC2EF0000E32EC1BF0400E32EC1BF01E
:10089000000E32EC1BF092EC2EF0000E32EC1BF04E
:1008A00087EF04F02942299E080E295E100E255C70
:1008B000D8B465EF04F092EC2EF0000E32EC1BF091
:1008C000000E32EC1BF06DEF04F04EEC2EF0000E3B
:1008D00032EC1BF0000E32EC1BF0295009EC20F03A
:1008E00055EC20F0400E32EC1BF0000E32EC1BF009
:1008F00025A082EF04F06EEC28F0000E32EC1BF025
:1009000087EF04F01EEC28F0000E32EC1BF0000E16
:1009100032EC1BF08EEC2CF0000E32EC1BF00EECE7
:100920002BF0000E32EC1BF07EEC21F0D9EC1AF02B
:10093000420EE2EC1AF0BC0E0AEC1BF0FEEC2AF0C0
:10094000000E32EC1BF072EC2EF0000E32EC1BF0BD
:100950002750296EFF0E295CD8A4D3EF04F04EEC8B
:100960002EF0000E32EC1BF0000E32EC1BF092EC7D
:100970002EF0000E32EC1BF092EC2EF0000E32EC5A
:100980001BF092EC2EF0000E32EC1BF0400E32EC1D
:100990001BF0000E32EC1BF092EC2EF0000E32EC4D
:1009A0001BF008EF05F02942299E080E295E100E63
:1009B000275CD8B4E6EF04F092EC2EF0000E32EC97
:1009C0001BF0000E32EC1BF0EEEF04F04EEC2EF0BC
:1009D000000E32EC1BF0000E32EC1BF0295009EC3B
:1009E00020F055EC20F0400E32EC1BF0000E32EC03
:1009F0001BF027A003EF05F06EEC28F0000E32ECA0
:100A00001BF008EF05F01EEC28F0000E32EC1BF096
:100A1000000E32EC1BF08EEC2CF0000E32EC1BF0D2
:100A20000EEC2BF0000E32EC1BF07EEC21F0D6EC3D
:100A30001AF0410EE2EC1AF0BD0E0AEC1BF05EEC6F
:100A40002BF0000E32EC1BF072EC2EF0000E32ECAC
:100A50001BF02650296E299C000E265CD8B43BEF73
:100A600005F0000E32EC1BF082EC2EF0000E32ECA2
:100A70001BF043EF05F0000E32EC1BF04EEC2EF0B5
:100A8000000E32EC1BF02942299E299C295009ECCA
:100A900020F05BEC20F0400E32EC1BF0000E32EC4C
:100AA0001BF026AC63EF05F026A072EF05F08EEC8C
:100AB00028F0000E32EC1BF06EEC28F0000E32EC49
:100AC0001BF088EF05F026A07EEF05F06EEC28F015
:100AD000000E32EC1BF01EEC28F0000E32EC1BF086
:100AE00088EF05F03EEC28F0000E32EC1BF06EECC7
:100AF00028F0000E32EC1BF088EF05F01EEC28F019
:100B0000000E32EC1BF01EEC28F0000E32EC1BF055
:100B1000000E32EC1BF08EEC2CF0000E32EC1BF0D1
:100B20000EEC2BF0000E32EC1BF07EEC21F0D9EC39
:100B30001AF0420EE2EC1AF0BD0E0AEC1BF05EEC6D
:100B40002BF0000E32EC1BF072EC2EF0000E32ECAB
:100B50001BF02850296E299C000E285CD8B4BBEFEE
:100B600005F0000E32EC1BF082EC2EF0000E32ECA1
:100B70001BF0C3EF05F0000E32EC1BF04EEC2EF034
:100B8000000E32EC1BF02942299E299C295009ECC9
:100B900020F05BEC20F0400E32EC1BF0000E32EC4B
:100BA0001BF028ACE3EF05F028A0F2EF05F08EEC87
:100BB00028F0000E32EC1BF06EEC28F0000E32EC48
:100BC0001BF008EF06F028A0FEEF05F06EEC28F011
:100BD000000E32EC1BF01EEC28F0000E32EC1BF085
:100BE00008EF06F03EEC28F0000E32EC1BF06EEC45
:100BF00028F0000E32EC1BF008EF06F01EEC28F097
:100C0000000E32EC1BF01EEC28F0000E32EC1BF054
:100C1000000E32EC1BF08EEC2CF0000E32EC1BF0D0
:100C20000EEC2BF0000E32EC1BF07EEC21F0D9EC38
:100C30001AF0400EE2EC1AF0B90E0AEC1BF036A0E6
:100C40003BEF06F0FF0E32EC1BF06EEC2DF0FF0ECA
:100C500032EC1BF0EEEC2DF0FF0E32EC1BF0DEEC74
:100C60002DF0FF0E32EC1BF0EEEC2CF0FF0E32EC10
:100C70001BF052EF06F0000E32EC1BF04EEC2EF0A3
:100C8000000E32EC1BF04EEC2EF0000E32EC1BF09E
:100C90004EEC2EF0000E32EC1BF04EEC2EF0000E5F
:100CA00032EC1BF036BA7EEC21F0D6EC1AF0400E96
:100CB000E2EC1AF0B90E0AEC1BF036B297EF06F030
:100CC000FF0E32EC1BF02EEC2DF0FF0E32EC1BF081
:100CD0007EEC2DF0FF0E32EC1BF0DEEC2DF0FF0E63
:100CE00032EC1BF0EEEC2CF0FF0E32EC1BF0BEEC05
:100CF0002DF0FF0E32EC1BF05EEC2DF0FF0E32EC0F
:100D00001BF08EEC2DF0FF0E32EC1BF0CEEC2CF035
:100D1000FF0E32EC1BF04EEC2DF0FF0E32EC1BF010
:100D20004EEC2EF0000E32EC1BF0D6EF06F0FF0E6C
:100D300032EC1BF0CEEC2DF0FF0E32EC1BF0EEECA3
:100D40002CF0FF0E32EC1BF09EEC2DF0FF0E32EC7F
:100D50001BF0AEEC2CF0FF0E32EC1BF0BEEC2DF0D5
:100D6000FF0E32EC1BF0AEEC2CF0FF0E32EC1BF061
:100D7000DEEC2DF0FF0E32EC1BF0EEEC2CF0FF0E53
:100D800032EC1BF05EEC2EF0FF0E32EC1BF036A4C2
:100D9000D1EF06F0BEEC2DF0FF0E32EC1BF0D6EFDB
:100DA00006F05EEC2DF0FF0E32EC1BF07EEC21F035
:100DB000D6EC1AF0400EE2EC1AF0BA0E0AEC1BF078
:100DC00036B61AEF07F0FF0E32EC1BF07EEC2DF07A
:100DD000FF0E32EC1BF08EEC2DF0FF0E32EC1BF010
:100DE000BEEC2DF0FF0E32EC1BF06EEC2DF0FF0E82
:100DF00032EC1BF0AEEC2CF0FF0E32EC1BF05EEC94
:100E00002DF0FF0E32EC1BF04EEC2EF0000E32EC0B
:100E10001BF04EEC2EF0000E32EC1BF04EEC2EF0E0
:100E2000000E32EC1BF04EEC2EF0000E32EC1BF0FC
:100E300089EF07F036B854EF07F0FF0E32EC1BF0E5
:100E4000AEEC2CF0FF0E32EC1BF0DEEC2DF0FF0EC2
:100E500032EC1BF0DEEC2DF0FF0E32EC1BF0EEEC72
:100E60002CF0FF0E32EC1BF07EEC2DF0FF0E32EC7E
:100E70001BF0EEEC2DF0FF0E32EC1BF0AEEC2CF084
:100E8000FF0E32EC1BF0DEEC2DF0FF0E32EC1BF00F
:100E90008EEC2DF0FF0E32EC1BF0BEEC2DF0FF0EB1
:100EA00032EC1BF089EF07F0FF0E32EC1BF0AEECDA
:100EB0002CF0FF0E32EC1BF06EEC2DF0FF0E32EC3E
:100EC0001BF09EEC2DF0FF0E32EC1BF05EEC2DF0D3
:100ED000FF0E32EC1BF02EEC2DF0FF0E32EC1BF06F
:100EE000FEEC2CF0FF0E32EC1BF02EEC2DF0FF0E82
:100EF00032EC1BF0EEEC2CF0FF0E32EC1BF0BEECF3
:100F00002DF0FF0E32EC1BF04EEC2EF0000E32EC0A
:100F10001BF07EEC21F0D9EC1AF0400EE2EC1AF056
:100F2000BA0E0AEC1BF036B8EDEF07F036BAB3EFA5
:100F300007F0FF0E32EC1BF0BEEC28F0FF0E32EC97
:100F40001BF0BF0E32EC1BF0FF0E32EC1BF00EEC70
:100F500029F0FF0E32EC1BF0BEEC28F0FF0E32EC55
:100F60001BF0CBEF07F0FF0E32EC1BF0BEEC28F0CD
:100F7000FF0E32EC1BF0BF0E32EC1BF0FF0E32EC1A
:100F80001BF0DEEC28F0FF0E32EC1BF00EEC29F02B
:100F9000FF0E32EC1BF0FF0E32EC1BF09EEC2CF03F
:100FA000FF0E32EC1BF0BEEC2CF05EEC2EF0CEEC23
:100FB0002DF0FF0E32EC1BF0DEEC2DF0FF0E32ECCC
:100FC0001BF0EEEC2CF0FF0E32EC1BF09EEC2DF043
:100FD000FF0E32EC1BF025EF08F0000E32EC1BF098
:100FE0004EEC2EF0000E32EC1BF0000E32EC1BF03B
:100FF000000E32EC1BF04EEC2EF0000E32EC1BF02B
:101000004EEC2EF0000E32EC1BF0000E32EC1BF01A
:101010004EEC2EF0000E32EC1BF04EEC2EF04EECAF
:101020002EF04EEC2EF0000E32EC1BF04EEC2EF0BB
:10103000000E32EC1BF04EEC2EF0000E32EC1BF0EA
:101040004EEC2EF0000E32EC1BF07EEC21F0D6ECD4
:101050001AF0400EE2EC1AF0BE0E0AEC1BF09EEC09
:101060002BF0000E32EC1BF0000E32EC1BF0C2EC49
:101070002EF001EC27F039503B6E3A503C6E3B06A7
:10108000000E2F5CD8A455EF08F040B051EF08F0E7
:10109000000E3B5ED8A451EF08F0C2EC2EF058EFE2
:1010A00008F0CCEC2EF058EF08F0C2EC2EF02F0632
:1010B000332A120E335CD8A43FEF08F0336A36BAF5
:1010C0007EEC21F0D9EC1AF0400EE2EC1AF0BE0EE4
:1010D0000AEC1BF03B06000E2F5CD8A480EF08F052
:1010E00040B07CEF08F0000E3B5ED8A47CEF08F027
:1010F000C2EC2EF083EF08F0CCEC2EF083EF08F07A
:10110000C2EC2EF02F06332A150E335CD8A46AEFFA
:1011100008F0336A7EEC21F0D6EC1AF0400EE2ECD7
:101120001AF0BF0E0AEC1BF0FEEC2BF0000E32ECB6
:101130001BF0000E32EC1BF0C2EC2EF03C06000E51
:101140002E5CD8A4B4EF08F040B0B0EF08F0000E69
:101150003C5ED8A4B0EF08F0C2EC2EF0B7EF08F078
:10116000CCEC2EF0B7EF08F0C2EC2EF02E06332AAE
:10117000120E335CD8A49EEF08F0336A36BA7EECC8
:1011800021F0D9EC1AF0400EE2EC1AF0BF0E0AEC96
:101190001BF03C06000E2E5CD8A4DFEF08F040B038
:1011A000DBEF08F0000E3C5ED8A4DBEF08F0C2ECE9
:1011B0002EF0E2EF08F0CCEC2EF0E2EF08F0C2ECFB
:1011C0002EF02E06332A150E335CD8A4C9EF08F092
:1011D000336A53EF01F07EEC21F080BE3EEF09F060
:1011E0000C0E465CD8B4F8EF08F0462A40EF09F040
:1011F000466A11B240EF09F0118212B00BEF09F00C
:10120000020E195CD8A408EF09F0196A40EF09F042
:10121000192A40EF09F0000E195CD8B42EEF09F03E
:10122000010E195CD8B41EEF09F03FAA1BEF09F0BC
:101230003F9A40EF09F03F8A40EF09F03FA62BEFBD
:1012400009F03FA828EF09F03F963F9840EF09F0DA
:101250003F8840EF09F03F8640EF09F03FA23BEFA7
:1012600009F03FA438EF09F03F923F9440EF09F0B6
:101270003F8440EF09F03F8240EF09F01192466A47
:1012800080BC92EF09F00C0E455CD8B44BEF09F02E
:10129000452A94EF09F0456A11B494EF09F01184DE
:1012A00012B05FEF09F0000E195CD8A45CEF09F0F2
:1012B000020E196E94EF09F0190694EF09F0000E72
:1012C000195CD8B482EF09F0010E195CD8B472EF42
:1012D00009F03FAA6FEF09F03F9A94EF09F03F8AB7
:1012E00094EF09F03FA67EEF09F03FA87BEF09F0ED
:1012F0003F9894EF09F03F9694EF09F03F863F88BE
:1013000094EF09F03FA28EEF09F03FA48BEF09F0B4
:101310003F9494EF09F03F9294EF09F03F823F84AD
:1013200094EF09F01194456A36BA7EEC21F0D6ECC0
:101330001AF0410EE2EC1AF0B80E0AEC1BF0700E37
:1013400032EC1BF0100E32EC1BF0100E32EC1BF0E6
:10135000100E32EC1BF0000E32EC1BF0AEEC2BF05A
:10136000000E32EC1BF02EEC2CF0000E32EC1BF0D9
:101370000EEC2CF0000E32EC1BF03EEC2BF0000ECD
:1013800032EC1BF00EEC2CF0000E32EC1BF08EEC6D
:1013900028F0000E32EC1BF03EEC28F0000E32EC90
:1013A0001BF04EEC28F0000E32EC1BF03EEC28F067
:1013B000000E32EC1BF03C0E32EC1BF0420E32EC15
:1013C0001BF0420E32EC1BF0420E32EC1BF0D9EC5B
:1013D0001AF0400EE2EC1AF0B80E0AEC1BF03C0ECC
:1013E00032EC1BF04EEC2EF00EEC2CF0000E32EC3A
:1013F0001BF03EEC2BF0000E32EC1BF01EEC2CF040
:10140000000E32EC1BF01EEC2CF0000E32EC1BF048
:101410007EEC2BF0000E32EC1BF0BEEC2BF0000E3D
:1014200032EC1BF05EEC2BF0000E32EC1BF0082AC5
:101430000F0E085CD8B422EF0AF0100E32EC1BF04D
:1014400017EF0AF0086A700E32EC1BF07EEC21F008
:10145000D6EC1AF0400EE2EC1AF0B90E0AEC1BF0D2
:1014600012B038EF0AF0000E195CD8B485EF0AF01C
:10147000000E32EC1BF09EEC2BF0000E32EC1BF059
:10148000000E32EC1BF0A2EC2EF0000E32EC1BF042
:10149000000E32EC1BF0FEEC2BF04EEC2EF01EECAE
:1014A0002BF0000E32EC1BF06EEC2BF04EEC2EF01D
:1014B0001EEC2BF0000E32EC1BF0CEEC2BF0000EED
:1014C00032EC1BF0BEEC2BF0000E32EC1BF01EECED
:1014D0002CF0D9EC1AF0400EE2EC1AF0B90E0AEC3E
:1014E0001BF0000E32EC1BF0FEEC2BF0000E32EC89
:1014F0001BF0CEEC2BF0000E32EC1BF09EEC2BF030
:10150000000E32EC1BF0D0EF0AF0FF0E32EC1BF0B5
:101510005EEC2DF0FF0E32EC1BF0FF0E32EC1BF0F8
:10152000B2EC2EF0FF0E32EC1BF0FF0E32EC1BF093
:10153000BEEC2DF05EEC2EF0CEEC2CF0FF0E32EC7B
:101540001BF01EEC2DF05EEC2EF0CEEC2CF0FF0E1E
:1015500032EC1BF08EEC2DF0FF0E32EC1BF07EEC2B
:101560002DF0FF0E32EC1BF0DEEC2DF0D9EC1AF072
:10157000400EE2EC1AF0B90E0AEC1BF0FF0E32EC52
:101580001BF0BEEC2DF0FF0E32EC1BF08EEC2DF0BC
:10159000FF0E32EC1BF05EEC2DF0FF0E32EC1BF078
:1015A0007EEC21F0D6EC1AF0400EE2EC1AF0BB0E05
:1015B0000AEC1BF012B0E2EF0AF0010E195CD8B48D
:1015C00049EF0BF0000E32EC1BF0FEEC2AF0000E9F
:1015D00032EC1BF01EEC2CF0000E32EC1BF01EEC7B
:1015E0002CF0000E32EC1BF0A2EC2EF0000E32ECD0
:1015F0001BF0000E32EC1BF05EEC2BF0000E32EC18
:101600001BF0FEEC2AF0000E32EC1BF07EEC2BF00F
:10161000000E32EC1BF0BEEC2BF04EEC2EF01EEC6C
:101620002BF0000E32EC1BF03C0E32EC1BF0420EA5
:1016300032EC1BF0420E32EC1BF0420E32EC1BF08F
:10164000D9EC1AF0400EE2EC1AF0BB0E0AEC1BF0DB
:101650003C0E32EC1BF0000E32EC1BF0BEEC2BF01B
:10166000000E32EC1BF01EEC2CF0000E32EC1BF0E6
:10167000FEEC2BF0000E32EC1BF0CEEC2BF0000E4B
:1016800032EC1BF09EEC2BF0000E32EC1BF0AEEFB8
:101690000BF0FF0E32EC1BF0AEEC2CF0FF0E32EC38
:1016A0001BF0DEEC2DF0FF0E32EC1BF0DEEC2DF02B
:1016B000FF0E32EC1BF0B2EC2EF0FF0E32EC1BF002
:1016C000FF0E32EC1BF00EEC2DF0FF0E32EC1BF097
:1016D000AEEC2CF0FF0E32EC1BF02EEC2DF0FF0EDA
:1016E00032EC1BF07EEC2DF05EEC2EF0CEEC2CF00C
:1016F000FF0E32EC1BF0C30E32EC1BF0BD0E32ECD1
:101700001BF0BD0E32EC1BF0BD0E32EC1BF0D9EC21
:101710001AF0400EE2EC1AF0BB0E0AEC1BF0C30EFE
:1017200032EC1BF0FF0E32EC1BF07EEC2DF0FF0EC6
:1017300032EC1BF0DEEC2DF0FF0E32EC1BF0BEECB9
:101740002DF0FF0E32EC1BF08EEC2DF0FF0E32EC84
:101750001BF05EEC2DF0FF0E32EC1BF07EEC21F066
:10176000D6EC1AF0400EE2EC1AF0BD0E0AEC1BF0BB
:1017700012B0C0EF0BF0020E195CD8B41FEF0CF0E2
:10178000000E32EC1BF0FEEC2AF0000E32EC1BF0E7
:101790001EEC2CF0000E32EC1BF01EEC2CF0000EB8
:1017A00032EC1BF03EEC2BF0000E32EC1BF0BEECEA
:1017B0002BF0000E32EC1BF02EEC2CF0000E32EC75
:1017C0001BF0FEEC2AF0000E32EC1BF01EEC2CF0AD
:1017D000000E32EC1BF0CEEC2BF0000E32EC1BF0C6
:1017E000FEEC2BF0000E32EC1BF0000E32EC1BF086
:1017F000000E32EC1BF0000E32EC1BF0D9EC1AF0AC
:10180000400EE2EC1AF0BD0E0AEC1BF0000E32ECBA
:101810001BF00EEC2CF0000E32EC1BF01EEC2CF04A
:10182000000E32EC1BF03EEC2BF0000E32EC1BF005
:10183000DEEC2BF0000E32EC1BF07CEF0CF0FF0E18
:1018400032EC1BF0AEEC2CF0FF0E32EC1BF0DEECB9
:101850002DF0FF0E32EC1BF0DEEC2DF0FF0E32EC23
:101860001BF0EEEC2CF0FF0E32EC1BF07EEC2DF0BA
:10187000FF0E32EC1BF0EEEC2DF0FF0E32EC1BF005
:10188000AEEC2CF0FF0E32EC1BF0DEEC2DF0FF0E78
:1018900032EC1BF08EEC2DF0FF0E32EC1BF0BEECA8
:1018A0002DF0FF0E32EC1BF0FF0E32EC1BF0FF0EA2
:1018B00032EC1BF0FF0E32EC1BF0D9EC1AF0400EAC
:1018C000E2EC1AF0BD0E0AEC1BF0FF0E32EC1BF03E
:1018D000CEEC2DF0FF0E32EC1BF0DEEC2DF0FF0E07
:1018E00032EC1BF0EEEC2CF0FF0E32EC1BF09EEC19
:1018F0002DF0FF0E32EC1BF07EEC21F0D6EC1AF04E
:10190000430EE2EC1AF0BA0E0AEC1BF01E0E32EC9B
:101910001BF0100E32EC1BF0100E32EC1BF0100E10
:1019200032EC1BF0100E32EC1BF0D6EC1AF0430E2A
:10193000E2EC1AF0BC0E0AEC1BF01E0E32EC1BF0AF
:10194000100E32EC1BF0100E32EC1BF0100E32ECCD
:101950001BF0100E32EC1BF0D6EC1AF0430EE2EC4A
:101960001AF0BE0E0AEC1BF01E0E32EC1BF0100E2D
:1019700032EC1BF0100E32EC1BF0100E32EC1BF0B0
:10198000100E32EC1BF0D6EC1AF04A0EE2EC1AF014
:10199000BA0E0AEC1BF03FB24EEF0DF012A0D6EFDC
:1019A0000CF0000E195CD8B412EF0DF0000E32EC02
:1019B0001BF07EEC2BF0000E32EC1BF0BEEC2BF09B
:1019C000000E32EC1BF01EEC2CF0000E32EC1BF083
:1019D0003EEC2BF0000E32EC1BF0FEEC2BF0000E78
:1019E00032EC1BF09EEC2BF0000E32EC1BF0CEEC38
:1019F0002BF0000E32EC1BF01EEC2BF0000E32EC44
:101A00001BF08EEC2BF0D9EC1AF0400EE2EC1AF041
:101A1000BA0E0AEC1BF0000E32EC1BF04EEC2EF06E
:101A2000E0EF0DF0FF0E32EC1BF02EEC2DF0FF0E70
:101A300032EC1BF07EEC2DF0FF0E32EC1BF0DEECF6
:101A40002DF0FF0E32EC1BF0EEEC2CF0FF0E32EC22
:101A50001BF0BEEC2DF0FF0E32EC1BF05EEC2DF017
:101A6000FF0E32EC1BF08EEC2DF0FF0E32EC1BF073
:101A7000CEEC2CF0FF0E32EC1BF04EEC2DF0D9EC3E
:101A80001AF0400EE2EC1AF0BA0E0AEC1BF0FF0E50
:101A900032EC1BF04EEC2EF0E0EF0DF012A056EF02
:101AA0000DF0000E195CD8B49CEF0DF0000E32EC76
:101AB0001BF00EEC2CF0000E32EC1BF03EEC2BF089
:101AC000000E32EC1BF0DEEC2BF0000E32EC1BF0C3
:101AD000FEEC2AF0000E32EC1BF0FEEC2BF0000EB8
:101AE00032EC1BF0FEEC2AF0000E32EC1BF01EEC88
:101AF0002CF0000E32EC1BF03EEC2BF0000E32EC22
:101B00001BF04EEC2EF0D9EC1AF0400EE2EC1AF07D
:101B1000BA0E0AEC1BF03FA495EF0DF0FEEC2BF093
:101B2000000E32EC1BF0E0EF0DF09EEC2BF0000EFF
:101B300032EC1BF0E0EF0DF0FF0E32EC1BF0CEECC0
:101B40002DF0FF0E32EC1BF0EEEC2CF0FF0E32EC21
:101B50001BF09EEC2DF0FF0E32EC1BF0AEEC2CF0E7
:101B6000FF0E32EC1BF0BEEC2DF0FF0E32EC1BF042
:101B7000AEEC2CF0FF0E32EC1BF0DEEC2DF0FF0E85
:101B800032EC1BF0EEEC2CF0FF0E32EC1BF05EECB6
:101B90002EF0D9EC1AF0400EE2EC1AF0BA0E0AEC74
:101BA0001BF03FA4DBEF0DF0BEEC2DF0FF0E32EC8E
:101BB0001BF0E0EF0DF05EEC2DF0FF0E32EC1BF0B1
:101BC0007EEC21F0D6EC1AF04A0EE2EC1AF0BC0ED4
:101BD0000AEC1BF03FB673EF0EF012A0F5EF0DF01C
:101BE000010E195CD8B434EF0EF0000E32EC1BF08D
:101BF000BEEC2BF0000E32EC1BF0CEEC2BF0000E06
:101C000032EC1BF0FEEC2BF0000E32EC1BF0AEECD5
:101C10002BF0000E32EC1BF0FEEC2AF0000E32EC42
:101C20001BF09EEC2BF0000E32EC1BF04EEC2EF075
:101C3000000E32EC1BF04EEC2EF0000E32EC1BF0DE
:101C40004EEC2EF0D9EC1AF0400EE2EC1AF0BC0E7D
:101C50000AEC1BF0000E32EC1BF04EEC2EF0000EE6
:101C600032EC1BF080EF0FF0FF0E32EC1BF07EEC3D
:101C70002DF0FF0E32EC1BF08EEC2DF0FF0E32EC4F
:101C80001BF0BEEC2DF0FF0E32EC1BF06EEC2DF0D5
:101C9000FF0E32EC1BF0AEEC2CF0FF0E32EC1BF022
:101CA0005EEC2DF0FF0E32EC1BF04EEC2EF0000E31
:101CB00032EC1BF04EEC2EF0000E32EC1BF04EEC32
:101CC0002EF0D9EC1AF0400EE2EC1AF0BC0E0AEC41
:101CD0001BF0000E32EC1BF04EEC2EF0000E32EC3E
:101CE0001BF080EF0FF03FB8FCEF0EF012A07EEF7C
:101CF0000EF0010E195CD8B4BDEF0EF0000E32EC00
:101D00001BF0FEEC2AF0000E32EC1BF01EEC2CF067
:101D1000000E32EC1BF01EEC2CF0000E32EC1BF02F
:101D20003EEC2BF0000E32EC1BF0BEEC2BF0000E64
:101D300032EC1BF02EEC2CF0000E32EC1BF0FEEC23
:101D40002AF0000E32EC1BF01EEC2CF0000E32ECF0
:101D50001BF0CEEC2BF0D9EC1AF0400EE2EC1AF0AE
:101D6000BC0E0AEC1BF0000E32EC1BF0FEEC2BF06C
:101D7000000E32EC1BF080EF0FF0FF0E32EC1BF088
:101D8000AEEC2CF0FF0E32EC1BF0DEEC2DF0FF0E73
:101D900032EC1BF0DEEC2DF0FF0E32EC1BF0EEEC23
:101DA0002CF0FF0E32EC1BF07EEC2DF0FF0E32EC2F
:101DB0001BF0EEEC2DF0FF0E32EC1BF0AEEC2CF035
:101DC000FF0E32EC1BF0DEEC2DF0FF0E32EC1BF0C0
:101DD0008EEC2DF0D9EC1AF0400EE2EC1AF0BC0EAD
:101DE0000AEC1BF0FF0E32EC1BF0BEEC2DF0FF0EE8
:101DF00032EC1BF080EF0FF012A004EF0FF0010E99
:101E0000195CD8B443EF0FF0000E32EC1BF0FEEC7F
:101E10002AF0000E32EC1BF0AEEC2BF0000E32EC90
:101E20001BF0DEEC2BF0000E32EC1BF09EEC2BF0E6
:101E3000000E32EC1BF07EEC2BF0000E32EC1BF0AF
:101E40004EEC2BF0000E32EC1BF07EEC2BF0000E73
:101E500032EC1BF03EEC2BF0000E32EC1BF0FEECF3
:101E60002BF0D9EC1AF0400EE2EC1AF0BC0E0AECA2
:101E70001BF0000E32EC1BF04EEC2EF0000E32EC9C
:101E80001BF080EF0FF0FF0E32EC1BF0AEEC2CF0ED
:101E9000FF0E32EC1BF06EEC2DF0FF0E32EC1BF05F
:101EA0009EEC2DF0FF0E32EC1BF05EEC2DF0FF0EE1
:101EB00032EC1BF02EEC2DF0FF0E32EC1BF0FEECA2
:101EC0002CF0FF0E32EC1BF02EEC2DF0FF0E32EC5E
:101ED0001BF0EEEC2CF0FF0E32EC1BF0BEEC2DF004
:101EE000D9EC1AF0400EE2EC1AF0BC0E0AEC1BF032
:101EF000FF0E32EC1BF04EEC2EF0000E32EC1BF01D
:101F00007EEC21F0D6EC1AF04A0EE2EC1AF0BE0E8E
:101F10000AEC1BF03FBAE3EF0FF012A095EF0FF0C1
:101F2000020E195CD8B4BCEF0FF0000E32EC1BF0BF
:101F30001EEC28F0000E32EC1BF0400E32EC1BF0D1
:101F4000000E32EC1BF06EEC28F0000E32EC1BF0B1
:101F50001EEC28F0000E32EC1BF0000E32EC1BF0F1
:101F60008EEC2CF0000E32EC1BF00EEC2BF0000E81
:101F700032EC1BF037EF10F0FF0E32EC1BF0BEEC32
:101F800028F0FF0E32EC1BF0BF0E32EC1BF0FF0E00
:101F900032EC1BF00EEC29F0FF0E32EC1BF0BEEC25
:101FA00028F0FF0E32EC1BF0FF0E32EC1BF09EEC23
:101FB0002CF0FF0E32EC1BF0BEEC2CF0FF0E32ECDE
:101FC0001BF037EF10F012A0EBEF0FF0020E195CD0
:101FD000D8B412EF10F0000E32EC1BF01EEC28F01B
:101FE000000E32EC1BF0400E32EC1BF0000E32EC17
:101FF0001BF03EEC28F0000E32EC1BF06EEC28F0EB
:10200000000E32EC1BF0000E32EC1BF08EEC2CF0CC
:10201000000E32EC1BF00EEC2BF0000E32EC1BF03D
:1020200037EF10F0FF0E32EC1BF0BEEC28F0FF0E85
:1020300032EC1BF0BF0E32EC1BF0FF0E32EC1BF04B
:10204000DEEC28F0FF0E32EC1BF00EEC29F0FF0E58
:1020500032EC1BF0FF0E32EC1BF09EEC2CF0FF0E6E
:1020600032EC1BF0BEEC2CF0FF0E32EC1BF053EF09
:1020700001F07EEC21F080BE81EF10F00C0E465C8A
:10208000D8B446EF10F0462A83EF10F0466A11B23A
:1020900083EF10F0118212B259EF10F0020E1A5CA9
:1020A000D8A456EF10F01A6A83EF10F01A2A83EFC3
:1020B00010F0000E1A5CD8A467EF10F041A064EF96
:1020C00010F0419083EF10F0418083EF10F0010E8B
:1020D0001A5CD8B478EF10F0000E4B5CD8A475EF02
:1020E00010F0020E4B6E83EF10F04B0683EF10F0F2
:1020F00041A27EEF10F0419283EF10F0418283EF16
:1021000010F01192466A80BCC9EF10F00C0E455CCD
:10211000D8B48EEF10F0452ACBEF10F0456A11B419
:10212000CBEF10F0118412B2A2EF10F0000E1A5C87
:10213000D8A49FEF10F0020E1A6ECBEF10F01A0623
:10214000CBEF10F0000E1A5CD8A4B0EF10F041A055
:10215000ADEF10F04190CBEF10F04180CBEF10F0DD
:10216000010E1A5CD8B4C0EF10F0020E4B5CD8A47C
:10217000BDEF10F04B6ACBEF10F04B2ACBEF10F015
:1021800041A2C6EF10F04192CBEF10F04182CBEFAD
:1021900010F01194456A36BA7EEC21F0D6EC1AF0B4
:1021A000410EE2EC1AF0B80E0AEC1BF0700E32ECA5
:1021B0001BF0100E32EC1BF0100E32EC1BF0100E68
:1021C00032EC1BF0000E32EC1BF0CEEC2BF0000ECC
:1021D00032EC1BF01EEC2CF0000E32EC1BF06EEC1F
:1021E0002BF0000E32EC1BF03EEC2BF0000E32EC2C
:1021F0001BF0FEEC2BF04EEC2EF00EEC2CF0000E53
:1022000032EC1BF03EEC2BF0000E32EC1BF01EEC1F
:102210002CF0000E32EC1BF01EEC2CF0D9EC1AF076
:10222000400EE2EC1AF0B80E0AEC1BF07EEC2BF03C
:10223000000E32EC1BF0BEEC2BF0000E32EC1BF06B
:102240005EEC2BF0000E32EC1BF0082A2D0E085C21
:10225000D8B430EF11F0100E32EC1BF025EF11F076
:10226000086A700E32EC1BF07EEC21F0D6EC1AF00E
:10227000400EE2EC1AF0B90E0AEC1BF012B246EF77
:1022800011F0000E1A5CD8B472EF11F0000E32ECAF
:102290001BF0DEEC2BF0000E32EC1BF03EEC2BF0D2
:1022A000000E32EC1BF0FEEC2AF0000E32EC1BF0BC
:1022B0008EEC2BF04EEC2EF06EEC2BF0000E32EC90
:1022C0001BF0CEEC2BF0000E32EC1BF09EEC2BF052
:1022D000000E32EC1BF02EEC2BF0000E32EC1BF05B
:1022E0009CEF11F0FF0E32EC1BF09EEC2DF0FF0E78
:1022F00032EC1BF0EEEC2CF0FF0E32EC1BF0AEECEF
:102300002CF0FF0E32EC1BF04EEC2DF05EEC2EF0BC
:102310001EEC2DF0FF0E32EC1BF08EEC2DF0FF0EBC
:1023200032EC1BF05EEC2DF0FF0E32EC1BF0DEEC1D
:102330002CF0FF0E32EC1BF0D6EC1AF0430EE2EC60
:102340001AF0BA0E0AEC1BF01E0E32EC1BF0100E47
:1023500032EC1BF0100E32EC1BF0100E32EC1BF0C6
:10236000100E32EC1BF036BA7EEC21F0D6EC1AF0EF
:10237000400EE2EC1AF0BD0E0AEC1BF012B2C6EFF2
:1023800011F0020E1A5CD8B41EEF12F0000E32ECFF
:102390001BF09EEC2BF0000E32EC1BF03EEC2BF011
:1023A000000E32EC1BF03EEC2CF0000E32EC1BF079
:1023B0003EEC2BF0000E32EC1BF09EEC2BF04EECC2
:1023C0002EF0AEEC2BF0000E32EC1BF01EEC2CF0DD
:1023D0004EEC2EF0FEEC2BF0000E32EC1BF01EEC5F
:1023E0002CF0000E32EC1BF0000E32EC1BF0D9EC9E
:1023F0001AF0400EE2EC1AF0BD0E0AEC1BF0000ED3
:1024000032EC1BF0000E32EC1BF0000E32EC1BF035
:102410001EEC2CF0000E32EC1BF07EEC2BF0000ECC
:1024200032EC1BF0AEEC2BF0000E32EC1BF03EEC6D
:102430002BF0000E32EC1BF074EF12F0FF0E32ECBA
:102440001BF05EEC2DF0FF0E32EC1BF0EEEC2CF0EE
:10245000FF0E32EC1BF0FEEC2DF0FF0E32EC1BF009
:10246000EEEC2CF0FF0E32EC1BF05EEC2DF05EEC8F
:102470002EF06EEC2DF0FF0E32EC1BF0DEEC2DF0AA
:102480005EEC2EF0BEEC2DF0FF0E32EC1BF0DEEC1D
:102490002DF0FF0E32EC1BF0FF0E32EC1BF0D9ECEE
:1024A0001AF0400EE2EC1AF0BD0E0AEC1BF0FF0E23
:1024B00032EC1BF0FF0E32EC1BF0FF0E32EC1BF087
:1024C000DEEC2DF0FF0E32EC1BF02EEC2DF0FF0EAB
:1024D00032EC1BF06EEC2DF0FF0E32EC1BF0EEEC4C
:1024E0002CF0FF0E32EC1BF0D6EC1AF0430EE2ECAF
:1024F0001AF0BE0E0AEC1BF01E0E32EC1BF0100E92
:1025000032EC1BF0100E32EC1BF0100E32EC1BF014
:10251000100E32EC1BF07EEC21F0D6EC1AF0400EDF
:10252000E2EC1AF0BB0E0AEC1BF012B29DEF12F0B7
:10253000010E1A5CD8B4CEEF12F0000E32EC1BF094
:10254000DEEC2BF0000E32EC1BF03EEC2BF0000E1C
:1025500032EC1BF0FEEC2AF0000E32EC1BF08EEC9D
:102560002BF04EEC2EF0FEEC2BF0000E32EC1BF0BC
:102570003EEC2BF0000E32EC1BF00EEC2CF0000EBB
:1025800032EC1BF03EEC2BF0000E32EC1BF01EEC9C
:102590002CF0000E32EC1BF0FDEF12F0FF0E32ECCF
:1025A0001BF09EEC2DF0FF0E32EC1BF0EEEC2CF04D
:1025B000FF0E32EC1BF0AEEC2CF0FF0E32EC1BF0F9
:1025C0004EEC2DF05EEC2EF0BEEC2DF0FF0E32EC5A
:1025D0001BF0EEEC2CF0FF0E32EC1BF0CEEC2DF0ED
:1025E000FF0E32EC1BF0EEEC2CF0FF0E32EC1BF089
:1025F000DEEC2DF0FF0E32EC1BF07EEC21F0D6EC81
:102600001AF0430EE2EC1AF0BC0E0AEC1BF01E0EA0
:1026100032EC1BF0100E32EC1BF0100E32EC1BF003
:10262000100E32EC1BF0100E32EC1BF0D6EC1AF050
:102630004A0EE2EC1AF0BA0E0AEC1BF041B05BEF66
:1026400013F0000E1A5CD8A429EF13F012B242EF77
:1026500013F0000E32EC1BF06EEC2BF0000E32EC9F
:102660001BF0CEEC2BF0000E32EC1BF09EEC2BF0AE
:10267000000E32EC1BF02EEC2BF0000E32EC1BF0B7
:1026800093EF13F0FF0E32EC1BF01EEC2DF0FF0E5B
:1026900032EC1BF08EEC2DF0FF0E32EC1BF05EECFA
:1026A0002DF0FF0E32EC1BF0DEEC2CF0FF0E32ECC6
:1026B0001BF093EF13F0000E1A5CD8A463EF13F035
:1026C00012B27CEF13F0000E32EC1BF04EEC2BF04C
:1026D000000E32EC1BF0FEEC2BF0000E32EC1BF087
:1026E0003EEC2BF0000E32EC1BF03EEC2BF0000E1B
:1026F00032EC1BF093EF13F0FF0E32EC1BF0FEEC0C
:102700002CF0FF0E32EC1BF0BEEC2DF0FF0E32EC85
:102710001BF0EEEC2CF0FF0E32EC1BF0EEEC2CF08C
:10272000FF0E32EC1BF036BA7EEC21F0D6EC1AF03C
:102730004A0EE2EC1AF0BE0E0AEC1BF0000E4B5CE7
:10274000D8B4F6EF13F0010E4B5CD8B444EF14F09C
:10275000020E1A5CD8A4B0EF13F012B2D3EF13F04C
:10276000000E32EC1BF00EEC2CF0000E32EC1BF0E5
:102770009EEC2BF0000E32EC1BF0CEEC2BF0000E9A
:1027800032EC1BF04EEC2CF0000E32EC1BF04EEC59
:102790002EF0000E32EC1BF04EEC2EF0000E32EC60
:1027A0001BF090EF14F0FF0E32EC1BF0CEEC2DF08E
:1027B000FF0E32EC1BF05EEC2DF0FF0E32EC1BF046
:1027C0008EEC2DF0FF0E32EC1BF00EEC2EF0FF0E17
:1027D00032EC1BF04EEC2EF0000E32EC1BF04EEC07
:1027E0002EF0000E32EC1BF090EF14F0020E1A5C8B
:1027F000D8A4FEEF13F012B221EF14F0000E32EC69
:102800001BF04EEC2BF0000E32EC1BF0FEEC2AF02D
:10281000000E32EC1BF00EEC2CF0000E32EC1BF034
:102820001EEC2CF0000E32EC1BF04EEC2EF0000EE5
:1028300032EC1BF04EEC2EF0000E32EC1BF090EF61
:1028400014F0FF0E32EC1BF0FEEC2CF0FF0E32EC1D
:102850001BF0AEEC2CF0FF0E32EC1BF0CEEC2DF0AA
:10286000FF0E32EC1BF0DEEC2DF0FF0E32EC1BF015
:102870004EEC2EF0000E32EC1BF04EEC2EF0000E63
:1028800032EC1BF090EF14F0020E1A5CD8A44CEF5F
:1028900014F012B26FEF14F0000E32EC1BF0BEEC2D
:1028A0002BF0000E32EC1BF0CEEC2BF0000E32ECD5
:1028B0001BF0FEEC2BF0000E32EC1BF0AEEC2BF01C
:1028C000000E32EC1BF0FEEC2AF0000E32EC1BF096
:1028D0009EEC2BF0000E32EC1BF090EF14F0FF0E8C
:1028E00032EC1BF07EEC2DF0FF0E32EC1BF08EEC88
:1028F0002DF0FF0E32EC1BF0BEEC2DF0FF0E32EC93
:102900001BF06EEC2DF0FF0E32EC1BF0AEEC2CF059
:10291000FF0E32EC1BF05EEC2DF0FF0E32EC1BF0E4
:102920007EEC21F0D6EC1AF04A0EE2EC1AF0BC0E66
:102930000AEC1BF041B2FFEF14F0010E1A5CD8A4B0
:10294000A5EF14F012B2D2EF14F0000E32EC1BF02F
:102950001EEC2CF0000E32EC1BF07EEC2BF0000E87
:1029600032EC1BF0AEEC2BF0000E32EC1BF03EEC28
:102970002BF04EEC2EF0CEEC2BF0000E32EC1BF0D8
:102980002EEC2CF0000E32EC1BF01EEC2CF0000EA6
:1029900032EC1BF0000E32EC1BF0000E32EC1BF0A0
:1029A0005FEF15F0FF0E32EC1BF0DEEC2DF0FF0EAA
:1029B00032EC1BF02EEC2DF0FF0E32EC1BF06EEC27
:1029C0002DF0FF0E32EC1BF0EEEC2CF05EEC2EF056
:1029D0008EEC2DF0FF0E32EC1BF0EEEC2DF0FF0E26
:1029E00032EC1BF0DEEC2DF0FF0E32EC1BF0000E93
:1029F00032EC1BF0000E32EC1BF05FEF15F0010E15
:102A00001A5CD8A407EF15F012B234EF15F0000EDF
:102A100032EC1BF02EEC2BF0000E32EC1BF03EECF7
:102A20002BF0000E32EC1BF01EEC2BF0000E32EC03
:102A30001BF0FEEC2BF0000E32EC1BF03EEC2BF00A
:102A4000000E32EC1BF0FEEC2AF0000E32EC1BF014
:102A50000EEC2CF0000E32EC1BF03EEC2BF0000ED6
:102A600032EC1BF05FEF15F0FF0E32EC1BF0DEECEA
:102A70002CF0FF0E32EC1BF0EEEC2CF0FF0E32ECE3
:102A80001BF0CEEC2CF0FF0E32EC1BF0BEEC2DF068
:102A9000FF0E32EC1BF0EEEC2CF0FF0E32EC1BF0D4
:102AA000AEEC2CF0FF0E32EC1BF0CEEC2DF0FF0E56
:102AB00032EC1BF0EEEC2CF0FF0E32EC1BF07EEC57
:102AC00021F0D6EC1AF0460EE2EC1AF0BF0E0AEC3A
:102AD0001BF00EEC2CF0000E32EC1BF0CEEC2BF0C9
:102AE000000E32EC1BF04EEC2BF0000E32EC1BF023
:102AF0001EEC2CF0000E32EC1BF04EEC2CF0000E15
:102B000032EC1BF0FEEC2AF0000E32EC1BF0FEEC77
:102B10002BF0000E32EC1BF03EEC2BF0000E32ECF2
:102B20001BF04EEC2EF03EEC2CF0D9EC1AF0400EDF
:102B3000E2EC1AF0BF0E0AEC1BF0000E32EC1BF0B8
:102B40003EEC2BF0000E32EC1BF0FEEC2BF0000EF6
:102B500032EC1BF00EEC2CF0000E32EC1BF07EEC95
:102B60002BF0000E32EC1BF0CEEC2BF0000E32EC12
:102B70001BF0BEEC2BF0000E32EC1BF04EEC2EF0F6
:102B8000000E32EC1BF02EEC28F0000E32EC1BF0A5
:102B9000000E32EC1BF0400E32EC1BF0000E32EC5B
:102BA0001BF01EEC28F0000E32EC1BF01EEC28F09F
:102BB000000E32EC1BF053EF01F07EEC21F080BEF2
:102BC00022EF16F00C0E465CD8B4EAEF15F0462A58
:102BD00024EF16F0466A11B224EF16F0118212B4F7
:102BE000FDEF15F0020E1B5CD8A4FAEF15F01B6A7E
:102BF00024EF16F01B2A24EF16F0000E1B5CD8A45D
:102C00000BEF16F043A008EF16F0439024EF16F0F8
:102C1000438024EF16F0020E1B5CD8A419EF16F0C7
:102C200043A216EF16F0439224EF16F0438224EFEE
:102C300016F03FAC1FEF16F03F9C24EF16F03F8CD0
:102C400024EF16F01192466A80BC68EF16F00C0E65
:102C5000455CD8B42FEF16F0452A6AEF16F0456AA6
:102C600011B46AEF16F0118412B443EF16F0000E9F
:102C70001B5CD8A440EF16F0020E1B6E6AEF16F034
:102C80001B066AEF16F0000E1B5CD8A451EF16F07D
:102C900043A04EEF16F043906AEF16F043806AEFC0
:102CA00016F0020E1B5CD8A45FEF16F043A25CEF97
:102CB00016F043926AEF16F043826AEF16F03FACCB
:102CC00065EF16F03F9C6AEF16F03F8C6AEF16F046
:102CD0001194456A36BA7EEC21F0D6EC1AF0410E1A
:102CE000E2EC1AF0B80E0AEC1BF0700E32EC1BF09E
:102CF000100E32EC1BF0100E32EC1BF0100E32EC0A
:102D00001BF0000E32EC1BF03EEC2BF0000E32EC10
:102D10001BF03EEC2BF0000E32EC1BF0DEEC2BF047
:102D2000000E32EC1BF0FEEC2BF0000E32EC1BF030
:102D3000CEEC2BF0000E32EC1BF0AEEC2BF04EEC98
:102D40002EF04EEC2CF0000E32EC1BF0FEEC2BF0D3
:102D5000000E32EC1BF07EEC2BF0D9EC1AF0400E9A
:102D6000E2EC1AF0B80E0AEC1BF01EEC2CF0000E90
:102D700032EC1BF03EEC2BF0000E32EC1BF0082A7C
:102D8000330E085CD8B4CAEF16F0100E32EC1BF00C
:102D9000BFEF16F0086A700E32EC1BF07EEC21F0EB
:102DA000D6EC1AF0400EE2EC1AF0B90E0AEC1BF069
:102DB00012B4E0EF16F0000E1B5CD8B423EF17F04E
:102DC000000E32EC1BF03EEC2BF0000E32EC1BF050
:102DD0003EEC2BF0000E32EC1BF0DEEC2BF0000E84
:102DE00032EC1BF0FEEC2BF0000E32EC1BF0CEECC4
:102DF0002BF0000E32EC1BF0AEEC2BF04EEC2EF074
:102E00004EEC2CF0000E32EC1BF0FEEC2BF0000E22
:102E100032EC1BF07EEC2BF0000E32EC1BF01EECC3
:102E20002CF0D9EC1AF0400EE2EC1AF0B90E0AECD4
:102E30001BF0000E32EC1BF03EEC2BF0000E32ECDF
:102E40001BF064EF17F0FF0E32EC1BF0EEEC2CF0F1
:102E5000FF0E32EC1BF0EEEC2CF0FF0E32EC1BF010
:102E60009EEC2DF0FF0E32EC1BF0BEEC2DF0FF0EB1
:102E700032EC1BF08EEC2DF0FF0E32EC1BF06EEC02
:102E80002DF05EEC2EF00EEC2EF0FF0E32EC1BF06F
:102E9000BEEC2DF0FF0E32EC1BF02EEC2DF0FF0EF1
:102EA00032EC1BF0DEEC2DF0D9EC1AF0400EE2EC27
:102EB0001AF0B90E0AEC1BF0FF0E32EC1BF0EEEC30
:102EC0002CF0FF0E32EC1BF0D6EC1AF0430EE2ECC5
:102ED0001AF0BA0E0AEC1BF01E0E32EC1BF0100EAC
:102EE00032EC1BF0100E32EC1BF0100E32EC1BF02B
:102EF000100E32EC1BF0D6EC1AF0400EE2EC1AF099
:102F0000BD0E0AEC1BF012B48BEF17F0020E1B5C27
:102F1000D8B4CEEF17F0000E32EC1BF02EEC2BF0F5
:102F2000000E32EC1BF03EEC2BF0000E32EC1BF0EE
:102F30004EEC2BF0000E32EC1BF0FEEC2AF0000EF3
:102F400032EC1BF02EEC2CF0000E32EC1BF09EEC61
:102F50002BF0000E32EC1BF01EEC2CF04EEC2EF0A1
:102F60009EEC2BF0000E32EC1BF0CEEC2BF0000EA2
:102F700032EC1BF0FEEC2AF0D9EC1AF0400EE2EC39
:102F80001AF0BD0E0AEC1BF0000E32EC1BF02EEC1A
:102F90002BF0000E32EC1BF00FEF18F0FF0E32ECAE
:102FA0001BF0DEEC2CF0FF0E32EC1BF0EEEC2CF004
:102FB000FF0E32EC1BF0FEEC2CF0FF0E32EC1BF09F
:102FC000AEEC2CF0FF0E32EC1BF0EEEC2DF0FF0E11
:102FD00032EC1BF05EEC2DF0FF0E32EC1BF0DEEC61
:102FE0002DF05EEC2EF05EEC2DF0FF0E32EC1BF0BF
:102FF0008EEC2DF0FF0E32EC1BF0AEEC2CF0D9EC89
:103000001AF0400EE2EC1AF0BD0E0AEC1BF0FF0EB7
:1030100032EC1BF0DEEC2CF0FF0E32EC1BF0D6ECA9
:103020001AF0430EE2EC1AF0BE0E0AEC1BF01E0E74
:1030300032EC1BF0100E32EC1BF0100E32EC1BF0D9
:10304000100E32EC1BF0100E32EC1BF0D6EC1AF026
:10305000400EE2EC1AF0BB0E0AEC1BF012B436EF95
:1030600018F0010E1B5CD8B4A0EF18F0000E32EC83
:103070001BF03EEC2CF0000E32EC1BF0CEEC2BF0F3
:10308000000E32EC1BF09EEC2BF04EEC2EF03EECE2
:103090002CF0000E32EC1BF0FEEC2AF0000E32ECAD
:1030A0001BF09EEC2BF0000E32EC1BF02EEC2CF003
:1030B000000E32EC1BF03EEC2BF04EEC2EF00EEC42
:1030C0002CF0000E32EC1BF0780E32EC1BF0D9EC39
:1030D0001AF0400EE2EC1AF0BB0E0AEC1BF0140ED4
:1030E00032EC1BF0120E32EC1BF0140E32EC1BF023
:1030F000780E32EC1BF0000E32EC1BF03EEC2CF0A4
:10310000000E32EC1BF03EEC2BF0000E32EC1BF00C
:103110004EEC2EF04EEC2BF0000E32EC1BF09EEC41
:103120002BF0000E32EC1BF0FEEC2AF0000E32EC1D
:103130001BF05EEC2BF0000E32EC1BF008EF19F0E8
:10314000FF0E32EC1BF0FEEC2DF0FF0E32EC1BF00C
:103150008EEC2DF0FF0E32EC1BF05EEC2DF05EECF1
:103160002EF0FEEC2DF0FF0E32EC1BF0AEEC2CF04E
:10317000FF0E32EC1BF05EEC2DF0FF0E32EC1BF07C
:10318000EEEC2DF0FF0E32EC1BF0EEEC2CF05EECD2
:103190002EF0CEEC2DF0FF0E32EC1BF0870E32EC51
:1031A0001BF0D9EC1AF0400EE2EC1AF0BB0E0AEC60
:1031B0001BF0EB0E32EC1BF0ED0E32EC1BF0EB0EC5
:1031C00032EC1BF0870E32EC1BF0FF0E32EC1BF0E2
:1031D000FEEC2DF0FF0E32EC1BF0EEEC2CF0FF0EAF
:1031E00032EC1BF05EEC2EF0FEEC2CF0FF0E32EC1D
:1031F0001BF05EEC2DF0FF0E32EC1BF0AEEC2CF071
:10320000FF0E32EC1BF00EEC2DF0FF0E32EC1BF03B
:10321000D6EC1AF0430EE2EC1AF0BC0E0AEC1BF0EE
:103220001E0E32EC1BF0100E32EC1BF0100E32ECC6
:103230001BF0100E32EC1BF0100E32EC1BF0D6EC33
:103240001AF04A0EE2EC1AF0BA0E0AEC1BF043B088
:1032500078EF19F0000E1B5CD8A432EF19F012B40D
:1032600055EF19F0000E32EC1BF01EEC2BF0000EA7
:1032700032EC1BF0FEEC2AF0000E32EC1BF0BEEC40
:103280002BF0000E32EC1BF01EEC2BF0000E32EC9B
:103290001BF03EEC2BF0000E32EC1BF09EEC2BF002
:1032A000000E32EC1BF0C4EF19F0FF0E32EC1BF0F5
:1032B000CEEC2CF0FF0E32EC1BF0AEEC2CF0FF0E3F
:1032C00032EC1BF07EEC2DF0FF0E32EC1BF0CEEC5E
:1032D0002CF0FF0E32EC1BF0EEEC2CF0FF0E32EC7B
:1032E0001BF05EEC2DF0FF0E32EC1BF0C4EF19F07A
:1032F000000E1B5CD8A480EF19F012B4A3EF19F0F4
:10330000000E32EC1BF04EEC2CF0000E32EC1BF0F9
:10331000FEEC2BF0000E32EC1BF07EEC2BF0000EDE
:1033200032EC1BF01EEC2CF0000E32EC1BF03EECED
:103330002BF0000E32EC1BF04EEC2EF0000E32ECB7
:103340001BF0C4EF19F0FF0E32EC1BF00EEC2EF068
:10335000FF0E32EC1BF0BEEC2DF0FF0E32EC1BF03A
:103360002EEC2DF0FF0E32EC1BF0DEEC2DF0FF0EFC
:1033700032EC1BF0EEEC2CF0FF0E32EC1BF04EECBE
:103380002EF0000E32EC1BF07EEC21F0D6EC1AF0A1
:103390004A0EE2EC1AF0BE0E0AEC1BF043B21FEF2D
:1033A0001AF0020E1B5CD8A4D9EF19F012B4FCEF8E
:1033B00019F0000E32EC1BF01EEC2BF0000E32EC7C
:1033C0001BF0FEEC2AF0000E32EC1BF0BEEC2BF0F2
:1033D000000E32EC1BF01EEC2BF0000E32EC1BF05A
:1033E0003EEC2BF0000E32EC1BF09EEC2BF0000EAE
:1033F00032EC1BF06BEF1AF0FF0E32EC1BF0CEEC50
:103400002CF0FF0E32EC1BF0AEEC2CF0FF0E32EC89
:103410001BF07EEC2DF0FF0E32EC1BF0CEEC2CF00E
:10342000FF0E32EC1BF0EEEC2CF0FF0E32EC1BF03A
:103430005EEC2DF0FF0E32EC1BF06BEF1AF0020E7B
:103440001B5CD8A427EF1AF012B44AEF1AF0000E52
:1034500032EC1BF09EEC2BF0000E32EC1BF0CEECAD
:103460002BF0000E32EC1BF0FEEC2AF0000E32ECDA
:103470001BF02EEC2BF0000E32EC1BF04EEC2EF07D
:10348000000E32EC1BF04EEC2EF0000E32EC1BF076
:103490006BEF1AF0FF0E32EC1BF05EEC2DF0FF0E1E
:1034A00032EC1BF08EEC2DF0FF0E32EC1BF0AEEC8C
:1034B0002CF0FF0E32EC1BF0DEEC2CF0FF0E32ECA9
:1034C0001BF04EEC2EF0000E32EC1BF04EEC2EF00A
:1034D000000E32EC1BF0D6EC1AF04A0EE2EC1AF0B9
:1034E000BC0E0AEC1BF03FBCA6EF1AF0010E1B5CF1
:1034F000D8A47EEF1AF012B492EF1AF0000E32EC5C
:103500001BF0CEEC2BF0000E32EC1BF04EEC2BF04F
:10351000000E32EC1BF04EEC2BF0000E32EC1BF0E8
:10352000D4EF1AF0FF0E32EC1BF08EEC2DF0FF0EF4
:1035300032EC1BF0FEEC2CF0FF0E32EC1BF0FEEC3C
:103540002CF0FF0E32EC1BF0D4EF1AF0010E1B5CD6
:10355000D8A4AEEF1AF012B4C2EF1AF0000E32EC9B
:103560001BF0CEEC2BF0000E32EC1BF0BEEC2BF07F
:10357000000E32EC1BF04EEC2EF0000E32EC1BF085
:10358000D4EF1AF0FF0E32EC1BF08EEC2DF0FF0E94
:1035900032EC1BF07EEC2DF0FF0E32EC1BF04EEC0B
:1035A0002EF0000E32EC1BF053EF01F08C888C9A59
:1035B00012008C988C8A12008C888C8A12008C984D
:1035C0008C9A1200016E5DEC1BF001508B6E8C9298
:1035D0008C900000000000000000000000000000CF
:1035E0000000000000008C840000000000000000CB
:1035F0000000000000000000000000008C940000AB
:1036000000000000000000000000000000000000BA
:1036100000001200026E5DEC1BF002508B6E8C926B
:103620008C9000000000000000000000000000007E
:103630000000000000008C8400000000000000007A
:103640000000000000000000000000008C9400005A
:10365000000000000000000000000000000000006A
:1036600000001200006E5DEC1BF012BE9BEC1BF024
:1036700000508B6E8C928C800000000000000000D7
:103680000000000000000000000000008C8400002A
:10369000000000000000000000000000000000002A
:1036A00000008C94000000000000000000000000FA
:1036B000000000000000000012000F01FF0E946ED9
:1036C00000018C828C9000000000000000000000CF
:1036D000000000000000000000008C8400000000DA
:1036E00000000000000000000000000000000000DA
:1036F00000000000000000000000000000000000CA
:10370000000000008C940000000000000000000099
:1037100000000000000000000000000000000000A9
:103720000000000081BE6DEF1BF08C920F01000EB7
:10373000946E00011200000E1F5CD8B4C0EF1BF0A5
:10374000010E1F5CD8B4D9EF1BF0020E1F5CD8B479
:10375000F0EF1BF0030E1F5CD8B405EF1CF0040E55
:103760001F5CD8B418EF1CF0050E1F5CD8B429EF0D
:103770001CF0060E1F5CD8B438EF1CF045EF1CF0AF
:103780001EB0CEEF1BF00042004200420042004259
:1037900000420042010E001645EF1CF000460046B4
:1037A00000460046004600460046800E001645EFE3
:1037B0001CF01EB0E6EF1BF0004200420042004247
:1037C00000420042030E001645EF1CF00046004682
:1037D0000046004600460046C00E001645EF1CF0AD
:1037E0001EB0FCEF1BF000420042004200420042CB
:1037F000070E001645EF1CF0004600460046004646
:103800000046E00E001645EF1CF01EB010EF1CF055
:1038100000420042004200420F0E001645EF1CF02D
:103820000046004600460046F00E001645EF1CF02C
:103830001EB022EF1CF00042004200421F0E001694
:1038400045EF1CF0004600460046F80E001645EF16
:103850001CF01EB032EF1CF0004200423F0E00167A
:1038600045EF1CF000460046FC0E001645EF1CF02C
:103870001EB040EF1CF000427F0E001645EF1CF01A
:103880000046FE0E001645EF1CF01200DCEC1AF0AC
:10389000400EE2EC1AF0B80E0AEC1BF0000E32EC0F
:1038A0001BF0012A800E015CD8A44EEF1CF0022A06
:1038B0000BEC1BF0400EE2EC1AF0C00E025CD8A438
:1038C0004EEF1CF01200106E000E105CD8A481EFB9
:1038D0001CF005B872EF1CF005BA76EF1CF07EEC18
:1038E00027F012004EEC2EF0058C120005BC7DEF87
:1038F0001CF0059C7EEC27F01200059C4EEC2EF08F
:103900001200010E105CD8A489EF1CF08EEC27F099
:103910001200020E105CD8A491EF1CF09EEC27F070
:103920001200030E105CD8A499EF1CF0AEEC27F047
:103930001200040E105CD8A4A1EF1CF0BEEC27F01E
:103940001200050E105CD8A4A9EF1CF0CEEC27F0F5
:103950001200060E105CD8A4B1EF1CF0DEEC27F0CC
:103960001200070E105CD8A4B9EF1CF0EEEC27F0A3
:103970001200080E105CD8A4C1EF1CF0FEEC27F07A
:1039800012000EEC28F01200106E000E105CD8A48D
:10399000CDEF1CF01EEC28F01200010E105CD8A434
:1039A000D5EF1CF02EEC28F01200020E105CD8A40B
:1039B000DDEF1CF03EEC28F01200030E105CD8A4E2
:1039C000E5EF1CF04EEC28F01200040E105CD8A4B9
:1039D000EDEF1CF05EEC28F01200050E105CD8A490
:1039E000F5EF1CF06EEC28F01200060E105CD8A467
:1039F000FDEF1CF07EEC28F01200070E105CD8A43E
:103A000005EF1DF08EEC28F01200080E105CD8A413
:103A10000DEF1DF09EEC28F01200AEEC28F0120025
:103A2000106E000E105CD8A419EF1DF0BEEC28F04B
:103A30001200010E105CD8A421EF1DF0CEEC28F08E
:103A40001200020E105CD8A429EF1DF0DEEC28F065
:103A50001200030E105CD8A431EF1DF0EEEC28F03C
:103A60001200040E105CD8A439EF1DF0FEEC28F013
:103A70001200050E105CD8A441EF1DF00EEC29F0E9
:103A80001200060E105CD8A449EF1DF01EEC29F0C0
:103A90001200070E105CD8A451EF1DF02EEC29F097
:103AA0001200080E105CD8A459EF1DF03EEC29F06E
:103AB00012004EEC29F01200062A0A0E065CD8A469
:103AC0005CEF1DF0066A1200062AFF0E065CD8A401
:103AD00064EF1DF0066A072A550E075CD8A464EF50
:103AE0001DF0066A076A1200062AFF0E065CD8A4BB
:103AF00074EF1DF0066A072AFF0E075CD8A474EF66
:103B00001DF0066A076A1200D6EC1AF0400EE2ECCD
:103B10001AF0BF0E0AEC1BF03EEC2CF0000E32EC5B
:103B20001BF0CEEC2BF0000E32EC1BF09EEC2BF0D9
:103B3000000E32EC1BF08EEC28F0000E32EC1BF085
:103B40003EEC28F0000E32EC1BF04EEC28F0000E9C
:103B500032EC1BF03EEC28F0000E32EC1BF01EECB9
:103B600028F04EEC2EF0FEEC2BF0000E32EC1BF0A9
:103B70003EEC2BF0D9EC1AF0400EE2EC1AF0BF0E3E
:103B80000AEC1BF03EEC2CF0000E32EC1BF0400E69
:103B900032EC1BF0000E32EC1BF02EEC28F0000E85
:103BA00032EC1BF0400E32EC1BF0000E32EC1BF03E
:103BB0001EEC28F0000E32EC1BF0400E036E7F0E60
:103BC000046ED6EC1AF00350E2EC1AF0BC0E0AECCC
:103BD0001BF0010E32EC1BF0D9EC1AF00450E2ECB1
:103BE0001AF0BC0E0AEC1BF0010E32EC1BF0032A9B
:103BF000040664EC1DF064EC1DF0800E035CD8A498
:103C0000E1EF1DF074EC1DF074EC1DF074EC1DF090
:103C100074EC1DF074EC1DF074EC1DF074EC1DF0F0
:103C200074EC1DF074EC1DF064EC1DF0400E036E9E
:103C30007F0E046ED6EC1AF00350E2EC1AF0BC0EC4
:103C40000AEC1BF0000E32EC1BF0D9EC1AF0045019
:103C5000E2EC1AF0BC0E0AEC1BF0000E32EC1BF08A
:103C6000032A040664EC1DF064EC1DF0800E035C76
:103C7000D8A41AEF1EF0128E74EC1DF074EC1DF037
:103C800074EC1DF074EC1DF074EC1DF074EC1DF080
:103C900074EC1DF064EC1DF01E80D6EC1AF04A0E98
:103CA000E2EC1AF0BB0E0AEC1BF0AEEC29F0000EB1
:103CB00032EC1BF0100E32EC1BF0100E32EC1BF04D
:103CC000100E32EC1BF0100E32EC1BF0100E32EC2A
:103CD0001BF0000E32EC1BF02EEC2AF0000E32EC42
:103CE0001BF04EEC2EF0000E32EC1BF09EEC29F097
:103CF000000E32EC1BF02EEC2AF0000E32EC1BF022
:103D0000BEEC29F0000E32EC1BF0DEEC29F0000EC8
:103D100032EC1BF02EEC2AF0000E32EC1BF0D9EC4A
:103D20001AF0400EE2EC1AF0BB0E0AEC1BF09EEC0F
:103D300029F0000E32EC1BF09EEC29F0000E32EC64
:103D40001BF06EEC2AF0000E32EC1BF0DEEC29F0DA
:103D5000000E32EC1BF02EEC2AF0000E32EC1BF0C1
:103D6000BEEC29F0000E32EC1BF01E90D6EC1AF0DF
:103D7000560EE2EC1AF0BC0E0AEC1BF05EEC29F0D9
:103D8000000E32EC1BF09EEC2AF0000E32EC1BF021
:103D90008EEC29F0000E32EC1BF0DEEC29F0000E68
:103DA00032EC1BF03EEC2AF0000E32EC1BF04EEC35
:103DB0002EF0000E32EC1BF00EEC2AF0000E32EC6E
:103DC0001BF0D9EC1AF0400EE2EC1AF0BC0E0AEC33
:103DD0001BF05EEC29F0000E32EC1BF06EEC29F0CB
:103DE000000E32EC1BF03EEC2AF0000E32EC1BF021
:103DF0006EEC2AF0000E32EC1BF05EEC29F0000EA7
:103E000032EC1BF08EEC2AF0000E32EC1BF03EEC94
:103E10002AF0000E32EC1BF06EEC2AF0000E32ECB1
:103E20001BF0DEEC2AF0000E32EC1BF01F2A080E0D
:103E30001F5CD8A43CEF1EF0129E1F6A74EC1DF0AC
:103E400074EC1DF074EC1DF074EC1DF074EC1DF0BE
:103E500074EC1DF074EC1DF074EC1DF074EC1DF0AE
:103E600074EC1DF074EC1DF074EC1DF074EC1DF09E
:103E700074EC1DF074EC1DF074EC1DF074EC1DF08E
:103E800074EC1DF074EC1DF074EC1DF074EC1DF07E
:103E900074EC1DF074EC1DF074EC1DF074EC1DF06E
:103EA00074EC1DF074EC1DF074EC1DF074EC1DF05E
:103EB00074EC1DF074EC1DF074EC1DF074EC1DF04E
:103EC00074EC1DF074EC1DF074EC1DF074EC1DF03E
:103ED00074EC1DF074EC1DF074EC1DF074EC1DF02E
:103EE00074EC1DF074EC1DF074EC1DF074EC1DF01E
:103EF00074EC1DF074EC1DF074EC1DF074EC1DF00E
:103F000074EC1DF074EC1DF074EC1DF074EC1DF0FD
:103F100074EC1DF074EC1DF074EC1DF074EC1DF0ED
:103F200074EC1DF074EC1DF074EC1DF074EC1DF0DD
:103F300074EC1DF074EC1DF074EC1DF074EC1DF0CD
:103F400074EC1DF074EC1DF074EC1DF074EC1DF0BD
:103F500074EC1DF074EC1DF074EC1DF074EC1DF0AD
:103F600074EC1DF074EC1DF074EC1DF074EC1DF09D
:103F700074EC1DF074EC1DF074EC1DF074EC1DF08D
:103F800074EC1DF074EC1DF074EC1DF074EC1DF07D
:103F900074EC1DF074EC1DF074EC1DF074EC1DF06D
:103FA00074EC1DF074EC1DF074EC1DF074EC1DF05D
:103FB00074EC1DF074EC1DF074EC1DF074EC1DF04D
:103FC00074EC1DF074EC1DF074EC1DF074EC1DF03D
:103FD00074EC1DF074EC1DF074EC1DF074EC1DF02D
:103FE00074EC1DF046EC1CF074EC1DF074EC1DF04C
:103FF00074EC1DF074EC1DF074EC1DF074EC1DF00D
:1040000074EC1DF074EC1DF074EC1DF074EC1DF0FC
:104010001200096E640E095ED8A012EF20F00A2A81
:104020000AEF20F0640E09260A0E095ED8A01CEFE4
:1040300020F00B2A14EF20F00A0E0926010E095E6B
:10404000D8A026EF20F00C2A1EEF20F012000D6EF3
:10405000100E0D5ED8A030EF20F00B2A28EF20F0D4
:10406000100E0D26010E0D5ED8A03AEF20F00C2A9E
:1040700032EF20F0120005880A5063EC1CF0000EAD
:1040800032EC1BF00598058A0B5063EC1CF0000E17
:1040900032EC1BF0059A0C5063EC1CF0000E32EC75
:1040A0001BF00A6A0B6A0C6A12000A50C4EC1CF07E
:1040B000000E32EC1BF00B50C4EC1CF0000E32EC86
:1040C0001BF00C50C4EC1CF0000E32EC1BF00A6A22
:1040D0000B6A0C6A12000A5010EC1DF0FF0E32EC55
:1040E0001BF00B5010EC1DF0FF0E32EC1BF00C50CF
:1040F00010EC1DF0FF0E32EC1BF00A6A0B6A0C6A22
:104100001200136E182A090E185CD8B497EF20F02D
:1041100013BE8FEF20F01EEC28F091EF20F02EEC74
:1041200028F0000E32EC1BF0134682EF20F0186AE4
:104130001200136E080E185CD8B4D6EF20F013BE30
:10414000BBEF20F018501C5CD8B4B1EF20F0000E8B
:1041500032EC1BF01EEC28F0000E32EC1BF0D2EF1C
:1041600020F0FF0E32EC1BF0BEEC28F0FF0E32EC1C
:104170001BF0D2EF20F018501C5CD8B4CAEF20F02E
:10418000000E32EC1BF02EEC28F0000E32EC1BF08F
:10419000D2EF20F0FF0E32EC1BF0CEEC28F0FF0E39
:1041A00032EC1BF0182A13469AEF20F0186A12001E
:1041B0008A94206E00000000000000000000000053
:1041C00000000000000000000000000000000000EF
:1041D0000000000000000000000000008A9220AEF5
:1041E000F5EF20F08A80F9EF20F08A9000000000BF
:1041F00000008A82000000000000000000000000B3
:1042000000000000000000000000000000000000AE
:104210000000000000000000000000008A92000082
:10422000000000000000000000000000000000008E
:104230000000000000000000000000002046212ACD
:10424000080E215CD8A4EFEF20F0216A22A02DEF08
:1042500021F0000E206E44EF21F022A234EF21F075
:10426000100E206E44EF21F022A43BEF21F0200E2F
:10427000206E44EF21F022A642EF21F0300E206E96
:1042800044EF21F0400E206E20AE4AEF21F08A80EC
:104290004EEF21F08A900000000000008A820000AA
:1042A000000000000000000000000000000000000E
:1042B00000000000000000000000000000000000FE
:1042C0000000000000008A920000000000000000D2
:1042D00000000000000000000000000000000000DE
:1042E0000000000000002046212A080E215CD8A40E
:1042F00044EF21F0216A8A828A84120080A884EF28
:1043000021F0238085EF21F0239080AA8BEF21F00C
:1043100023828CEF21F02392030E235CD8B4118CFE
:10432000000E235CD8A4A9EF21F011ACA9EF21F075
:10433000119C020E245CD8A4A2EF21F09CEC22F088
:10434000A9EF21F0010E245CD8A4A9EF21F0B0EC74
:1043500021F02350246EFF0E3D5CD8A43D2A1200AC
:1043600036BABCEF21F0190E3D5CD8B0BCEF21F09D
:104370000A0E3E6E03EF22F02D0E3D5CD8B0CCEF5E
:1043800021F036AAC8EF21F0140E3E6E03EF22F0A2
:10439000080E3E6E03EF22F0410E3D5CD8B0DCEF1C
:1043A00021F036AAD8EF21F00C0E3E6E03EF22F07A
:1043B000050E3E6E03EF22F0550E3D5CD8B0ECEFDB
:1043C00021F036AAE8EF21F0080E3E6E03EF22F04E
:1043D000030E3E6E03EF22F036AA01EF22F0690EC3
:1043E0003D5CD8B0F8EF21F0060E3E6E03EF22F0F0
:1043F0007D0E3D5CD8B001EF22F0030E3E6E03EF60
:1044000022F0010E3E6E3E50426E36B457EF22F05F
:1044100036B83AEF22F0100E255CD8B434EF22F013
:10442000FF0E255CD8A419EF22F025983D6A50EFC5
:1044300022F036AA27EF22F026BC24EF22F0268CA9
:10444000A8EC23F028EF22F0269CA8EC23F0250608
:1044500036A09DEC23F04206000E425CD8A408EF83
:1044600022F03D6A50EF22F036B83AEF22F036B62D
:1044700050EF22F02650296E299C3F0E295CD8A4CB
:1044800045EF22F03D6A50EF22F0262A36A0A8EC34
:1044900023F04206000E425CD8A408EF22F03D6AE9
:1044A0003E50426E36B457EF22F036B2120036B8A4
:1044B00086EF22F0100E275CD8B481EF22F0FF0EB9
:1044C000275CD8A467EF22F027983D6A120036AA2D
:1044D00075EF22F028BC72EF22F0288CA8EC23F0B4
:1044E00076EF22F0289CA8EC23F0270636A09DEC5E
:1044F00023F04206000E425CD8A457EF22F03D6A3A
:10450000120036B886EF22F036B612002850296E17
:10451000299C3F0E295CD8A490EF22F03D6A12003E
:10452000282A36A0A8EC23F04206000E425CD8A44C
:1045300057EF22F03D6A120036BAA8EF22F0190EAA
:104540003D5CD8B0A8EF22F00A0E3E6EEFEF22F0ED
:104550002D0E3D5CD8B0B8EF22F036AAB4EF22F0B1
:10456000140E3E6EEFEF22F0080E3E6EEFEF22F0DB
:10457000410E3D5CD8B0C8EF22F036AAC4EF22F05D
:104580000C0E3E6EEFEF22F0050E3E6EEFEF22F0C6
:10459000550E3D5CD8B0D8EF22F036AAD4EF22F009
:1045A000080E3E6EEFEF22F0030E3E6EEFEF22F0AC
:1045B00036AAEDEF22F0690E3D5CD8B0E4EF22F0B0
:1045C000060E3E6EEFEF22F07D0E3D5CD8B0EDEFB3
:1045D00022F0030E3E6EEFEF22F0010E3E6E3E50D3
:1045E000426E36B44EEF23F036B8FAEF22F036B60C
:1045F0000FEF23F02650296E299C000E295CD8B4B9
:104600000FEF23F0260636A0A8EC23F04206000E9A
:10461000425CD8A4F4EF22F03D6A47EF23F036B8AD
:1046200047EF23F0FF0E255CD8A41AEF23F03D6A74
:1046300047EF23F0EF0E255CD8A42EEF23F036AA27
:104640002AEF23F026AC2AEF23F0269CA8EC23F0D7
:1046500047EF23F025883D6A47EF23F036AA3CEF69
:1046600023F026AC39EF23F0269CA8EC23F03DEF95
:1046700023F0268CA8EC23F0252A36A09DEC23F00D
:104680004206000E425CD8A4F4EF22F03D6A3E5090
:10469000426E36B44EEF23F036B2120036B854EF05
:1046A00023F036B668EF23F02850296E299C000EBF
:1046B000295CD8B468EF23F0280636A0A8EC23F0D4
:1046C0004206000E425CD8A44EEF23F03D6A120071
:1046D00036B81200FF0E275CD8A471EF23F03D6AB4
:1046E0001200EF0E275CD8A483EF23F036AA80EFE8
:1046F00023F028AC80EF23F0289CA8EC23F01200D4
:1047000027883D6A120036AA91EF23F028AC8EEF7D
:1047100023F0289CA8EC23F092EF23F0288CA8EC3F
:1047200023F0272A36A09DEC23F04206000E425CBF
:10473000D8A44EEF23F03D6A1200226A2280255051
:10474000D8EC20F0226A22842750D8EC20F0120006
:10475000226A22822650D8EC20F0226A2286285033
:10476000D8EC20F01200226A2280000ED8EC20F053
:10477000226A2284000ED8EC20F0226A2282000EE7
:10478000D8EC20F0226A2286000ED8EC20F012002D
:104790002BB2CFEF23F02B1E030E2B162A1E2BB0AD
:1047A000FFEF24F0030E2A5CD8B0DBEF23F0000EFD
:1047B0002F6E37EF25F0050E2A5CD8B0E4EF23F01A
:1047C000010E2F6E37EF25F0070E2A5CD8B0EDEF03
:1047D00023F0020E2F6E37EF25F0080E2A5CD8B0BA
:1047E000F6EF23F0030E2F6E37EF25F0090E2A5C4B
:1047F000D8B0FFEF23F0040E2F6E37EF25F00A0E2E
:104800002A5CD8B008EF24F0050E2F6E37EF25F0A4
:104810000B0E2A5CD8B011EF24F0060E2F6E37EF86
:1048200025F00D0E2A5CD8B01AEF24F0070E2F6E7B
:1048300037EF25F00E0E2A5CD8B023EF24F0080ED7
:104840002F6E37EF25F0100E2A5CD8B02CEF24F035
:10485000090E2F6E37EF25F0120E2A5CD8B035EF17
:1048600024F00A0E2F6E37EF25F0140E2A5CD8B014
:104870003EEF24F00B0E2F6E37EF25F0170E2A5C5B
:10488000D8B047EF24F00C0E2F6E37EF25F0190E3D
:104890002A5CD8B050EF24F00D0E2F6E37EF25F0C4
:1048A0001D0E2A5CD8B059EF24F00E0E2F6E37EF94
:1048B00025F0200E2A5CD8B062EF24F00F0E2F6E88
:1048C00037EF25F0240E2A5CD8B06BEF24F0100EE1
:1048D0002F6E37EF25F0290E2A5CD8B074EF24F044
:1048E000110E2F6E37EF25F02E0E2A5CD8B07DEF1B
:1048F00024F0120E2F6E37EF25F0330E2A5CD8B05D
:1049000086EF24F0130E2F6E37EF25F0390E2A5C58
:10491000D8B08FEF24F0140E2F6E37EF25F0400E35
:104920002A5CD8B098EF24F0150E2F6E37EF25F0E3
:10493000490E2A5CD8B0A1EF24F0160E2F6E37EF87
:1049400025F0510E2A5CD8B0AAEF24F0170E2F6E76
:1049500037EF25F05B0E2A5CD8B0B3EF24F0180EC9
:104960002F6E37EF25F0660E2A5CD8B0BCEF24F02E
:10497000190E2F6E37EF25F0720E2A5CD8B0C5EFF6
:1049800024F01A0E2F6E37EF25F0800E2A5CD8B077
:10499000CEEF24F01B0E2F6E37EF25F0900E2A5C21
:1049A000D8B0D7EF24F01C0E2F6E37EF25F0A10EF4
:1049B0002A5CD8B0E0EF24F01D0E2F6E37EF25F003
:1049C000B50E2A5CD8B0E9EF24F01E0E2F6E37EF3B
:1049D00025F0CB0E2A5CD8B0F2EF24F01F0E2F6E1C
:1049E00037EF25F0E40E2A5CD8B0FBEF24F0200E60
:1049F0002F6E37EF25F0210E2F6E37EF25F0000ECA
:104A00002A5CD8A408EF25F0210E2F6E37EF25F091
:104A10001F0E2A5CD8B011EF25F0220E2F6E37EF53
:104A200025F0420E2A5CD8B01AEF25F0230E2F6E27
:104A300037EF25F06A0E2A5CD8B023EF25F0240E5C
:104A40002F6E37EF25F0960E2A5CD8B02CEF25F0AC
:104A5000250E2F6E37EF25F0C70E2A5CD8B035EF44
:104A600025F0260E2F6E37EF25F0270E2F6E2DB274
:104A70003EEF25F02D1E030E2D162C1E2DB06EEFD1
:104A800026F0030E2C5CD8B04AEF25F0000E2E6EF7
:104A9000A8EF26F0050E2C5CD8B053EF25F0010EE0
:104AA0002E6EA8EF26F0070E2C5CD8B05CEF25F038
:104AB000020E2E6EA8EF26F0080E2C5CD8B065EF23
:104AC00025F0030E2E6EA8EF26F0090E2C5CD8B050
:104AD0006EEF25F0040E2E6EA8EF26F00A0E2C5C69
:104AE000D8B077EF25F0050E2E6EA8EF26F00B0E4E
:104AF0002C5CD8B080EF25F0060E2E6EA8EF26F0C5
:104B00000D0E2C5CD8B089EF25F0070E2E6EA8EFA5
:104B100026F00E0E2C5CD8B092EF25F0080E2E6E0B
:104B2000A8EF26F0100E2C5CD8B09BEF25F0090EF4
:104B30002E6EA8EF26F0120E2C5CD8B0A4EF25F054
:104B40000A0E2E6EA8EF26F0140E2C5CD8B0ADEF36
:104B500025F00B0E2E6EA8EF26F0170E2C5CD8B0A9
:104B6000B6EF25F00C0E2E6EA8EF26F0190E2C5C79
:104B7000D8B0BFEF25F00D0E2E6EA8EF26F01D0E5B
:104B80002C5CD8B0C8EF25F00E0E2E6EA8EF26F0E4
:104B9000200E2C5CD8B0D1EF25F00F0E2E6EA8EFB2
:104BA00026F0240E2C5CD8B0DAEF25F0100E2E6E15
:104BB000A8EF26F0290E2C5CD8B0E3EF25F0110EFB
:104BC0002E6EA8EF26F02E0E2C5CD8B0ECEF25F060
:104BD000120E2E6EA8EF26F0330E2C5CD8B0F5EF37
:104BE00025F0130E2E6EA8EF26F0390E2C5CD8B0EF
:104BF000FEEF25F0140E2E6EA8EF26F0400E2C5C72
:104C0000D8B007EF26F0150E2E6EA8EF26F0490E4D
:104C10002C5CD8B010EF26F0160E2E6EA8EF26F002
:104C2000510E2C5CD8B019EF26F0170E2E6EA8EF9F
:104C300026F05B0E2C5CD8B022EF26F0180E2E6EFC
:104C4000A8EF26F0660E2C5CD8B02BEF26F0190EDC
:104C50002E6EA8EF26F0720E2C5CD8B034EF26F042
:104C60001A0E2E6EA8EF26F0800E2C5CD8B03DEF09
:104C700026F01B0E2E6EA8EF26F0900E2C5CD8B0FE
:104C800046EF26F01C0E2E6EA8EF26F0A10E2C5C2F
:104C9000D8B04FEF26F01D0E2E6EA8EF26F0B50E01
:104CA0002C5CD8B058EF26F01E0E2E6EA8EF26F022
:104CB000CB0E2C5CD8B061EF26F01F0E2E6EA8EF45
:104CC00026F0E40E2C5CD8B06AEF26F0200E2E6E93
:104CD000A8EF26F0210E2E6EA8EF26F0000E2C5C19
:104CE000D8A477EF26F0210E2E6EA8EF26F01F0E27
:104CF0002C5CD8B080EF26F0220E2E6EA8EF26F0A6
:104D0000420E2C5CD8B089EF26F0230E2E6EA8EF51
:104D100026F06A0E2C5CD8B092EF26F0240E2E6E90
:104D2000A8EF26F0960E2C5CD8B09BEF26F0250E4F
:104D30002E6EA8EF26F0C70E2C5CD8B0A4EF26F09C
:104D4000260E2E6EA8EF26F0270E2E6EA8EF26F068
:104D500031502F5CD8B0D1EF26F0000E315CD8B4C2
:104D6000D1EF26F0352A000E4A5CD8A4BBEF26F01E
:104D7000010EC4EF26F0010E4A5CD8A4C3EF26F062
:104D8000020EC4EF26F0030E355CD8A4CDEF26F05A
:104D9000310631502F6ED1EF26F031502F6ED2EF09
:104DA00026F0356A30502E5CD8B0FCEF26F0000EAD
:104DB000305CD8B4FCEF26F0342A000E4A5CD8A44C
:104DC000E5EF26F0010EEEEF26F0010E4A5CD8A4C6
:104DD000EDEF26F0020EEEEF26F0030E345CD8A4C1
:104DE000F7EF26F0300630502E6EFBEF26F03050F5
:104DF0002E6EFCEF26F0346A2F50316E2E50306E3E
:104E0000120040B22FEF27F03A502E5CD8A00EEFE0
:104E100027F02E503A6E386A19EF27F06E0E385C84
:104E2000D8B416EF27F0382A19EF27F0386A2E5039
:104E30003A6E39502F5CD8A023EF27F02F50396EEF
:104E4000376A2EEF27F06E0E375CD8B42BEF27F0C1
:104E5000372A2EEF27F0376A2F50396E12003A505A
:104E60002E5CD8A03AEF27F02E503A6E386A1E9288
:104E700056EF27F01EB245EF27F0460E385CD8B447
:104E800045EF27F0382A56EF27F0386A1E82000EC9
:104E90003A5CD8B456EF27F0080E4D5CD8B454EF06
:104EA00027F04D2A56EF27F04D6A3A0639502F5C0D
:104EB000D8A061EF27F02F50396E376A1E947DEF2E
:104EC00027F01EB46CEF27F0460E375CD8B46CEFB9
:104ED00027F0372A7DEF27F0376A1E84000E395CF1
:104EE000D8B47DEF27F0080E4C5CD8B47BEF27F0E8
:104EF0004C2A7DEF27F04C6A390612007C0E32EC0A
:104F00001BF0820E32EC1BF0820E32EC1BF0820E94
:104F100032EC1BF07C0E32EC1BF01200000E32EC77
:104F20001BF0840E32EC1BF0FE0E32EC1BF0800EF8
:104F300032EC1BF0000E32EC1BF01200E20E32ECF1
:104F40001BF0920E32EC1BF0920E32EC1BF0920E24
:104F500032EC1BF08C0E32EC1BF01200440E32ECE3
:104F60001BF0820E32EC1BF0920E32EC1BF0920E14
:104F700032EC1BF06C0E32EC1BF01200300E32ECF7
:104F80001BF0280E32EC1BF0240E32EC1BF0FE0E50
:104F900032EC1BF0200E32EC1BF012004E0E32EC05
:104FA0001BF08A0E32EC1BF08A0E32EC1BF08A0EDC
:104FB00032EC1BF0720E32EC1BF012007C0E32EC65
:104FC0001BF0920E32EC1BF0920E32EC1BF0920EA4
:104FD00032EC1BF0640E32EC1BF01200060E32ECC9
:104FE0001BF0020E32EC1BF0C20E32EC1BF0320E44
:104FF00032EC1BF00E0E32EC1BF012006C0E32EC99
:105000001BF0920E32EC1BF0920E32EC1BF0920E63
:1050100032EC1BF06C0E32EC1BF012004C0E32EC3A
:105020001BF0920E32EC1BF0920E32EC1BF0920E43
:1050300032EC1BF07C0E32EC1BF012003C0E32EC1A
:105040001BF0420E32EC1BF0420E32EC1BF0420E13
:1050500032EC1BF03C0E32EC1BF01200000E32EC76
:105060001BF0440E32EC1BF07E0E32EC1BF0400EB7
:1050700032EC1BF0000E32EC1BF01200720E32EC20
:105080001BF04A0E32EC1BF04A0E32EC1BF04A0EBB
:1050900032EC1BF0440E32EC1BF01200220E32EC0C
:1050A0001BF04A0E32EC1BF04A0E32EC1BF04A0E9B
:1050B00032EC1BF0340E32EC1BF01200300E32ECEE
:1050C0001BF0280E32EC1BF0240E32EC1BF07E0E8F
:1050D00032EC1BF0200E32EC1BF012002E0E32ECE4
:1050E0001BF04A0E32EC1BF04A0E32EC1BF04A0E5B
:1050F00032EC1BF0320E32EC1BF012003C0E32ECA4
:105100001BF04A0E32EC1BF04A0E32EC1BF04A0E3A
:1051100032EC1BF0300E32EC1BF01200060E32ECBB
:105120001BF0020E32EC1BF0620E32EC1BF0120E82
:1051300032EC1BF00E0E32EC1BF01200340E32EC8F
:105140001BF04A0E32EC1BF04A0E32EC1BF04A0EFA
:1051500032EC1BF0340E32EC1BF012000C0E32EC71
:105160001BF0520E32EC1BF0520E32EC1BF0520EC2
:1051700032EC1BF03C0E32EC1BF01200C30E32EC92
:105180001BF0BD0E32EC1BF0BD0E32EC1BF0BD0E61
:1051900032EC1BF0C30E32EC1BF01200FF0E32ECAF
:1051A0001BF0BB0E32EC1BF0810E32EC1BF0BF0E7D
:1051B00032EC1BF0FF0E32EC1BF012008D0E32ECC5
:1051C0001BF0B50E32EC1BF0B50E32EC1BF0B50E39
:1051D00032EC1BF0BB0E32EC1BF01200DD0E32EC99
:1051E0001BF0B50E32EC1BF0B50E32EC1BF0B50E19
:1051F00032EC1BF0CB0E32EC1BF01200CF0E32EC77
:105200001BF0D70E32EC1BF0DB0E32EC1BF0810EE4
:1052100032EC1BF0DF0E32EC1BF01200D10E32EC40
:105220001BF0B50E32EC1BF0B50E32EC1BF0B50ED8
:1052300032EC1BF0CD0E32EC1BF01200C30E32EC40
:105240001BF0B50E32EC1BF0B50E32EC1BF0B50EB8
:1052500032EC1BF0CF0E32EC1BF01200F90E32ECE8
:105260001BF0FD0E32EC1BF09D0E32EC1BF0ED0E30
:1052700032EC1BF0F10E32EC1BF01200CB0E32ECD4
:105280001BF0B50E32EC1BF0B50E32EC1BF0B50E78
:1052900032EC1BF0CB0E32EC1BF01200F30E32ECB2
:1052A0001BF0AD0E32EC1BF0AD0E32EC1BF0AD0E70
:1052B00032EC1BF0C30E32EC1BF01200F80E32EC95
:1052C0001BF0240E32EC1BF0220E32EC1BF0240EED
:1052D00032EC1BF0F80E32EC1BF01200FE0E32EC3A
:1052E0001BF0920E32EC1BF0920E32EC1BF0920E81
:1052F00032EC1BF06C0E32EC1BF012007C0E32EC28
:105300001BF0820E32EC1BF0820E32EC1BF0820E90
:1053100032EC1BF0440E32EC1BF01200FE0E32ECAD
:105320001BF0820E32EC1BF0820E32EC1BF0820E70
:1053300032EC1BF07C0E32EC1BF01200FE0E32EC55
:105340001BF0920E32EC1BF0920E32EC1BF0920E20
:1053500032EC1BF0820E32EC1BF01200FE0E32EC2F
:105360001BF0120E32EC1BF0120E32EC1BF0120E80
:1053700032EC1BF0020E32EC1BF012007C0E32EC11
:105380001BF0820E32EC1BF0820E32EC1BF0920E00
:1053900032EC1BF0740E32EC1BF01200FE0E32ECFD
:1053A0001BF0100E32EC1BF0100E32EC1BF0100E46
:1053B00032EC1BF0FE0E32EC1BF01200000E32EC51
:1053C0001BF0820E32EC1BF0FE0E32EC1BF0820E54
:1053D00032EC1BF0000E32EC1BF01200600E32ECCF
:1053E0001BF0800E32EC1BF0800E32EC1BF0800EB6
:1053F00032EC1BF07E0E32EC1BF01200FE0E32EC93
:105400001BF0100E32EC1BF0280E32EC1BF0440E99
:1054100032EC1BF0820E32EC1BF01200FE0E32EC6E
:105420001BF0800E32EC1BF0800E32EC1BF0800E75
:1054300032EC1BF0800E32EC1BF01200FE0E32EC50
:105440001BF0040E32EC1BF0080E32EC1BF0040EC5
:1054500032EC1BF0FE0E32EC1BF01200FE0E32ECB2
:105460001BF0080E32EC1BF0100E32EC1BF0200E7D
:1054700032EC1BF0FE0E32EC1BF012007C0E32EC14
:105480001BF0820E32EC1BF0820E32EC1BF0820E0F
:1054900032EC1BF07C0E32EC1BF01200FE0E32ECF4
:1054A0001BF0120E32EC1BF0120E32EC1BF0120E3F
:1054B00032EC1BF00C0E32EC1BF012007C0E32ECC6
:1054C0001BF0820E32EC1BF0A20E32EC1BF0420EEF
:1054D00032EC1BF0BC0E32EC1BF01200FE0E32EC74
:1054E0001BF0120E32EC1BF0120E32EC1BF0120EFF
:1054F00032EC1BF0EC0E32EC1BF012004C0E32ECD6
:105500001BF0920E32EC1BF0920E32EC1BF0920E5E
:1055100032EC1BF0640E32EC1BF01200020E32EC87
:105520001BF0020E32EC1BF0FE0E32EC1BF0020EF2
:1055300032EC1BF0020E32EC1BF012007E0E32EC4D
:105540001BF0800E32EC1BF0800E32EC1BF0800E54
:1055500032EC1BF07E0E32EC1BF012000E0E32EC21
:105560001BF0300E32EC1BF0C00E32EC1BF0300E94
:1055700032EC1BF00E0E32EC1BF012001E0E32EC61
:105580001BF0E00E32EC1BF0180E32EC1BF0E00EBC
:1055900032EC1BF01E0E32EC1BF01200C60E32EC89
:1055A0001BF0280E32EC1BF0100E32EC1BF0280E14
:1055B00032EC1BF0C60E32EC1BF012000E0E32EC79
:1055C0001BF0100E32EC1BF0E00E32EC1BF0100E54
:1055D00032EC1BF00E0E32EC1BF01200C20E32EC5D
:1055E0001BF0A20E32EC1BF0920E32EC1BF08A0E76
:1055F00032EC1BF0860E32EC1BF01200780E32EC0F
:105600001BF0140E32EC1BF0120E32EC1BF0140ED9
:1056100032EC1BF0780E32EC1BF012007E0E32ECF6
:105620001BF04A0E32EC1BF04A0E32EC1BF04A0E15
:1056300032EC1BF0340E32EC1BF012003C0E32EC5C
:105640001BF0420E32EC1BF0420E32EC1BF0420E0D
:1056500032EC1BF0240E32EC1BF012007E0E32EC0A
:105660001BF0420E32EC1BF0420E32EC1BF0420EED
:1056700032EC1BF03C0E32EC1BF012007E0E32ECD2
:105680001BF04A0E32EC1BF04A0E32EC1BF04A0EB5
:1056900032EC1BF0420E32EC1BF012007E0E32ECAC
:1056A0001BF00A0E32EC1BF00A0E32EC1BF00A0E55
:1056B00032EC1BF0020E32EC1BF012003C0E32EC0E
:1056C0001BF0420E32EC1BF0420E32EC1BF0520E7D
:1056D00032EC1BF0340E32EC1BF012007E0E32EC7A
:1056E0001BF0080E32EC1BF0080E32EC1BF0080E1B
:1056F00032EC1BF07E0E32EC1BF01200000E32EC8E
:105700001BF0420E32EC1BF07E0E32EC1BF0420E10
:1057100032EC1BF0000E32EC1BF012007E0E32EC6D
:105720001BF0100E32EC1BF0080E32EC1BF0140EC6
:1057300032EC1BF0620E32EC1BF012007E0E32ECEB
:105740001BF0400E32EC1BF0400E32EC1BF0400E12
:1057500032EC1BF0400E32EC1BF012007E0E32ECED
:105760001BF0040E32EC1BF0080E32EC1BF0040EA2
:1057700032EC1BF07E0E32EC1BF012007E0E32EC8F
:105780001BF0040E32EC1BF0180E32EC1BF0200E56
:1057900032EC1BF07E0E32EC1BF012003C0E32ECB1
:1057A0001BF0420E32EC1BF0420E32EC1BF0420EAC
:1057B00032EC1BF03C0E32EC1BF012007E0E32EC91
:1057C0001BF0120E32EC1BF0120E32EC1BF0120E1C
:1057D00032EC1BF00C0E32EC1BF012003C0E32ECE3
:1057E0001BF0420E32EC1BF0520E32EC1BF0220E7C
:1057F00032EC1BF05C0E32EC1BF012007E0E32EC31
:105800001BF0120E32EC1BF0120E32EC1BF0120EDB
:1058100032EC1BF06C0E32EC1BF01200440E32EC3A
:105820001BF04A0E32EC1BF04A0E32EC1BF04A0E13
:1058300032EC1BF0320E32EC1BF01200020E32EC96
:105840001BF0020E32EC1BF07E0E32EC1BF0020E4F
:1058500032EC1BF0020E32EC1BF012003E0E32EC6A
:105860001BF0400E32EC1BF0400E32EC1BF0400EF1
:1058700032EC1BF03E0E32EC1BF01200060E32EC46
:105880001BF0180E32EC1BF0600E32EC1BF0180E01
:1058900032EC1BF0060E32EC1BF012007E0E32ECE6
:1058A0001BF0200E32EC1BF0100E32EC1BF0200E21
:1058B00032EC1BF07E0E32EC1BF01200460E32EC86
:1058C0001BF0280E32EC1BF0100E32EC1BF0280EF1
:1058D00032EC1BF0460E32EC1BF01200060E32ECDE
:1058E0001BF0080E32EC1BF0700E32EC1BF0080EB1
:1058F00032EC1BF0060E32EC1BF01200440E32ECC0
:105900001BF0640E32EC1BF0540E32EC1BF04C0E0C
:1059100032EC1BF0440E32EC1BF01200300E32EC75
:105920001BF0480E32EC1BF0480E32EC1BF0480E18
:1059300032EC1BF07E0E32EC1BF01200CF0E32EC7C
:105940001BF0B70E32EC1BF0B70E32EC1BF0B70EAB
:1059500032EC1BF0810E32EC1BF01200870E32ECA1
:105960001BF0EB0E32EC1BF0ED0E32EC1BF0EB0EED
:1059700032EC1BF0870E32EC1BF01200810E32EC81
:105980001BF0B50E32EC1BF0B50E32EC1BF0B50E71
:1059900032EC1BF0CB0E32EC1BF01200C30E32ECDB
:1059A0001BF0BD0E32EC1BF0BD0E32EC1BF0BD0E39
:1059B00032EC1BF0DB0E32EC1BF01200810E32ECED
:1059C0001BF0BD0E32EC1BF0BD0E32EC1BF0BD0E19
:1059D00032EC1BF0C30E32EC1BF01200810E32ECE5
:1059E0001BF0B50E32EC1BF0B50E32EC1BF0B50E11
:1059F00032EC1BF0BD0E32EC1BF01200810E32ECCB
:105A00001BF0F50E32EC1BF0F50E32EC1BF0F50E30
:105A100032EC1BF0FD0E32EC1BF01200C30E32EC28
:105A20001BF0BD0E32EC1BF0BD0E32EC1BF0AD0EC8
:105A300032EC1BF0CB0E32EC1BF01200810E32EC7C
:105A40001BF0F70E32EC1BF0F70E32EC1BF0F70EEA
:105A500032EC1BF0810E32EC1BF01200FF0E32EC28
:105A60001BF0BD0E32EC1BF0810E32EC1BF0BD0EB4
:105A700032EC1BF0FF0E32EC1BF01200CF0E32ECBA
:105A80001BF0BF0E32EC1BF0BF0E32EC1BF0BF0E52
:105A900032EC1BF0C10E32EC1BF01200810E32EC26
:105AA0001BF0EF0E32EC1BF0F70E32EC1BF0EB0E9E
:105AB00032EC1BF09D0E32EC1BF01200810E32EC2A
:105AC0001BF0BF0E32EC1BF0BF0E32EC1BF0BF0E12
:105AD00032EC1BF0BF0E32EC1BF01200810E32ECE8
:105AE0001BF0FB0E32EC1BF0F70E32EC1BF0FB0E42
:105AF00032EC1BF0810E32EC1BF01200810E32EC06
:105B00001BF0FB0E32EC1BF0E70E32EC1BF0DF0E4D
:105B100032EC1BF0810E32EC1BF01200C30E32ECA3
:105B20001BF0BD0E32EC1BF0BD0E32EC1BF0BD0EB7
:105B300032EC1BF0C30E32EC1BF01200810E32EC83
:105B40001BF0ED0E32EC1BF0ED0E32EC1BF0ED0E07
:105B500032EC1BF0F30E32EC1BF01200C30E32ECF1
:105B60001BF0BD0E32EC1BF0AD0E32EC1BF0DD0E67
:105B700032EC1BF0A30E32EC1BF01200810E32EC63
:105B80001BF0ED0E32EC1BF0ED0E32EC1BF0ED0EC7
:105B900032EC1BF0930E32EC1BF01200BB0E32EC19
:105BA0001BF0B50E32EC1BF0B50E32EC1BF0B50E4F
:105BB00032EC1BF0CD0E32EC1BF01200FD0E32EC7D
:105BC0001BF0FD0E32EC1BF0810E32EC1BF0FD0ED3
:105BD00032EC1BF0FD0E32EC1BF01200C10E32EC69
:105BE0001BF0BF0E32EC1BF0BF0E32EC1BF0BF0EF1
:105BF00032EC1BF0C10E32EC1BF01200F90E32EC4D
:105C00001BF0E70E32EC1BF09F0E32EC1BF0E70EA0
:105C100032EC1BF0F90E32EC1BF01200810E32EC6C
:105C20001BF0DF0E32EC1BF0EF0E32EC1BF0DF0E40
:105C300032EC1BF0810E32EC1BF01200B90E32EC8C
:105C40001BF0D70E32EC1BF0EF0E32EC1BF0D70E30
:105C500032EC1BF0B90E32EC1BF01200F90E32ECF4
:105C60001BF0F70E32EC1BF08F0E32EC1BF0F70E30
:105C700032EC1BF0F90E32EC1BF01200000E32EC8D
:105C80001BF0000E32EC1BF0040E32EC1BF00A0E7F
:105C900032EC1BF0040E32EC1BF01200000E32EC62
:105CA0001BF0000E32EC1BF0000E32EC1BF0000E6D
:105CB00032EC1BF0000E32EC1BF01200FF0E32EC47
:105CC0001BF0FF0E32EC1BF0FF0E32EC1BF0FF0E50
:105CD00032EC1BF0FF0E32EC1BF01200280E32ECFF
:105CE0001BF01200280E32EC1BF0280E32EC1BF0D9
:105CF000280E32EC1BF0280E32EC1BF0280E32EC92
:105D00001BF01200100E32EC1BF0100E32EC1BF0E8
:105D10007C0E32EC1BF0100E32EC1BF0100E32EC4D
:105D20001BF01200100E32EC1BF0100E32EC1BF0C8
:105D3000100E32EC1BF0100E32EC1BF0100E32EC99
:105D40001BF01200400E32EC1BF0200E32EC1BF068
:105D5000100E32EC1BF0080E32EC1BF0040E32EC8D
:105D60001BF01200BF0E32EC1BF0DF0E32EC1BF00A
:105D7000EF0E32EC1BF0F70E32EC1BF0FB0E32ECA8
:105D80001BF012007E0E32EC1BF07E0E32EC1BF08C
:105D9000000E32EC1BF01200000E32EC1BF0000E75
:105DA00032EC1BF0000E32EC1BF01200000EAA6E5B
:105DB000000EA96E36BCEDEF2EF036A6E8EF2EF001
:105DC00036A8E8EF2EF03650E60BA86EF0EF2EF076
:105DD0003650EE0BA86EF0EF2EF03650FE0BA86E8C
:105DE000A69EA69CA684550EA76EAA0EA76EA68296
:105DF000A6B2F8EF2EF0A6941200000EAA6E010EC5
:105E0000A96E4050A86EA69EA69CA684550EA76EAD
:105E1000AA0EA76EA682A6B20BEF2FF0A6941200D0
:105E2000000EAA6E020EA96E4A50A86EA69EA69CEF
:105E3000A684550EA76EAA0EA76EA682A6B21EEF66
:105E40002FF0A6941200000EAA6E030EA96E255024
:105E5000A86EA69EA69CA684550EA76EAA0EA76E37
:105E6000A682A6B231EF2FF0A6941200000EAA6E01
:105E7000040EA96E2650A86EA69EA69CA684550E5A
:105E8000A76EAA0EA76EA682A6B244EF2FF0A69424
:105E90001200000EAA6E050EA96E2750A86EA69ECF
:105EA000A69CA684550EA76EAA0EA76EA682A6B2C1
:105EB00057EF2FF0A6941200000EAA6E060EA96EE0
:105EC0002850A86EA69EA69CA684550EA76EAA0E64
:0E5ED000A76EA682A6B26AEF2FF0A69412006B
:020000040030CA
:03000100381800AC
:02000500358044
:060008000FC00FE00F40E5
:0200000400F00A
:0400000000000100FB
:00000001FF
